:106D6E000000B30200000301FA0400EF0500030A5D
:106D7E000A5A0B001E0C00FA0D00030E00040F0140
:106D8E0064100096120132130AFA14010217010A56
:106D9E001801EF1905321A010A1B01EF1C05321FEB
:106DAE00FFFF20FFFF23011E2400642A00FA2B00A0
:106DBE00FA2C50782D003C2E00463000643250786C
:106DCE003300003432FA350164360164370150382D
:106DDE000A643A00033B00043C00643E003C3F0062
:106DEE000040FFFF411450420A5A430AC84405327C
:106DFE004500B44600FA4900024B00014C00FA501F
:106E0E000404510596520A32530B46540A965705FE
:106E1E0046590A465A32FA5B010A5C0A325E000A89
:106E2E005F00646200FE64FFFF67FFFF6801016997
:106E3E0001016A05966B00006C32966D00047300BA
:106E4E00017400017801327901327E0064810064A0
:106E5E0084FFFF8800028A00019D0A969E00019F12
:106E6E00FFFFA0FFFFA2000AA3FFFFA4FFFFA5FFE5
:106E7E00FFA6FFFFA7FFFFA8FFFFA9FFFF01010469
:106E8E001501022F003C4701044803045601044E2D
:106E9E00FFFF58000261FFFF6600028500AF86000B
:106EAE00018700FA89010A990008A100FAFAFAFA94
:106EBE000101021501022F1E3C470104480304562E
:106ECE0001034EFFFF58000261FFFF6600028500BE
:106EDE00AF8600018700FA89010A990000A100001F
:106EEE00FAFAFA0101021501022F1E3C470102486F
:106EFE0003035601014EFFFF58000061FFFF6600BD
:106F0E000085FFFF86FFFF87FFFF890102990000C2
:106F1E00A10000FAFAFA0065006F00790083008D77
:106F2E00009700A100AC00B600C000CA00D400DE7D
:106F3E0000E800F2005800600068007000780080E1
:106F4E0000880090009800A000A800B000B800C112
:106F5E0000C800D000D800DF00E600EE00F60041C9
:106F6E000047004D00530059005F0065006C007132
:106F7E000077007D00830089008F0095009B00A2A2
:106F8E0000A700AC00B200B900C000C500CA00D214
:0A6F9E0000D500DD00E100E700EF80
:103CD80085F97485FA757E017F00E5751270BAE57D
:103CE800742FFF50010E8E5A8F5B900014E0FCA3D6
:103CF800E0FDEF2DFDEE3CFC8C5C8D5D900034E02A
:103D0800FAA3E0FBED2BFBEC3AFA8A5C8B5D22759B
:103D1800A71085F97485FA757E017F00E575127024
:103D2800BAE5742FFF50010E8E5A8F5B9000DEE0CB
:103D3800B40210AC2DAD2EEF2DFDEE3CFC8C5C8D4D
:103D48005D8016AE5AAF5B900014E0FCA3E0FDEF77
:103D58002DFDEE3CFC8C5C8D5DAE5CAF5D9000345F
:103D6800E0FCA3E0FDEF2DFDEE3CFC8C5C8D5D22BC
:103D7800E55DF5FBE55CF5FCD29322E55DF5E9E54B
:103D88005CF5EAD29422E55DF5EBE55CF5ECD291C1
:103D980022E55DF5EDE55CF5EED2922275A710E51A
:103DA8005DF5FBE55CF5FC75A700D2872275A710C9
:103DB800E55DF5E9E55CF5EA75A700D2902275A7FF
:103DC80010E55DF5EBE55CF5EC75A700E5B544108D
:103DD800F5B52275A710E55DF5EDE55CF5EE75A77F
:103DE80000E5B54420F5B522E50C906921F82828AE
:103DF80073023EB675E700A239B34008E5B544083A
:103E0800F5B58006E5B554F7F5B575E710023EB689
:103E180075E700A239B34008E5B54402F5B5800658
:103E2800E5B554FDF5B575E710023EB6A23992A284
:103E3800807CA23992A1807675E700A239B3400848
:103E4800E5B54440F5B58006E5B554BFF5B575E769
:103E580010805B75E700A239B34008E5B54480F5EA
:103E6800B58006E5B5547FF5B575E7108040A239F1
:103E78009287803AA2399290803475E700A239B3CC
:103E88004008E5B54410F5B58006E5B554EFF5B53D
:103E980075E710801975E700A239B34008E5B54405
:0E3EA80020F5B58006E5B554DFF5B575E710D9
:10692100023DF9023DFC023E18023E34023E3A02AB
:106931003E40023E5B023E76023E7C023E82023EC9
:016941009DB8
:103EB60022743490014FF0742B900150F0743290BC
:103EC6000151F07448900152F0746F900153F074F0
:103ED6006D900154F07465900155F0742090015670
:103EE600F07434900157F07443900158F07479904F
:103EF6000159F0746C90015AF0742090015BF074D3
:103F06002090015CF0742090015DF022900886E01C
:103F1600FEA3E0FF741DD39F74019E400C906D6E4E
:103F2600120048E493F599804C90F802E493B405A6
:103F360014900886E0FEA3E0FF906DA1120048E40D
:103F460093F599803090F802E493D3940540149049
:103F56000886E0FEA3E0FF906D6E120048E493F53C
:103F6600998012900886E0FEA3E0FF906DD41200BF
:103F760048E493F5999008861270C8900886E0FE8A
:103F8600A3E0FFEFB45007EEB40103754E0022AE76
:103F96005AAF5B74B48E048F05FF1270AA8C5C8DC9
:103FA6005DAE5AAF5B74B48E048F05FF1270D58C6C
:103FB6005A8D5BC200E55B455A601374B4C3955BCA
:103FC600FFE4955AFE8E5A8F5B785C12710DE5748C
:103FD600A85CB80015D3955D4010E574C3955DFFE8
:103FE600E4955CFE8E5C8F5D8012E5742402C395B9
:103FF6005DFFE4955CFE8E5C8F5DD2002290008CA6
:10400600E0B40104C20A8002D20A90008DE0B40135
:1040160004C20B8002D20B9000CAE075F0D7A4FF51
:10402600AEF0740A8E048F05FF1270AA90087AEC1F
:10403600F0A3EDF09000CAE075F02BA4FFAEF0906F
:104046000010EEF0A3EFF07E017F00900088E012F2
:1040560070BA9000CBE08E048F05FF1270AA740A26
:10406600FF1270AA8D619000D4E075F0D7A4FFAE60
:10407600F0740A8E048F05FF1270AA90087EECF089
:10408600A3EDF09000D6E060139000D6E0F5F07452
:104096001684FF7E00EF9008DCF0800674649008BA
:1040A600DCF09000CCE0900066F0900118E0900003
:1040B60073F090011AE0FE9000C8E08E0088F0A42C
:1040C600FFAEF0EF9008E5F09000F3E075F013A472
:1040D600FDACF0900034ECF0A3EDF0A223B3401653
:1040E600900164E0700C900165E07006900166E056
:1040F60060028002C223900164E0B4300F90016533
:10410600E0B44708900166E0643B60028004D22474
:104116008002C22474E3900065F09000B5E0B40B11
:104126000874E3900065F0805A9000B5E0B4191267
:104136009000CBE0906F0F12008CE493900065F036
:1041460080419000B5E0B41E129000CBE0906F2D38
:1041560012008CE493900065F080289000B5E0B4DE
:1041660028129000CBE0906F5712008CE4939000D9
:1041760065F0800F9000B5E0B446089000ACE09082
:104186000065F0900085E0FE9008E6E06E601A7526
:1041960099E612019C74AB90003FF012069A7509DD
:1041A600647508001205E480FE90007DE0700674D8
:1041B600009000B2F090006AE0FE9000B2E0B50612
:1041C6006390006DE0FE9000D0E0B5065790006B5E
:1041D600E0FE9000DEE0B5064B900071E0FE900038
:1041E60085E0B5063F90006EE0FE9000C0E0B506A3
:1041F6003390006CE0FE9000CEE0B5062790006F8D
:10420600E0FE9000EBE0B5061B900070E0FE90002B
:10421600ECE0B5060F900072E0FE9000FEE06E70D6
:104226000302449B90008DE070089000CEE0640489
:104236006002800674039000CEF0900047E0C394BD
:104246000550087402900101F080149000DEE060D1
:10425600087406900101F08006740A900101F0903E
:104266000085E0B401067400900085F0900085E0BA
:10427600B4020674009000D0F0900085E0B4030606
:1042860074009000DDF09000D0E0D39401402774D4
:104296001B900103F074009006CEF074009006CFD8
:1042A600F0740090009AF09000B2E0B40206740137
:1042B6009000B2F080339000B2E0B4021A7400901D
:1042C6000103F074009006CEF074009006CFF074EF
:1042D6001B90009AF080127400900103F0741B90FA
:1042E60006CEF0740090009AF09000B2E06014746C
:1042F6001C900099F074009006D2F074009006D3DA
:10430600F0800C7400900099F0741C9006D2F09026
:1043160000EBE060147419900105F074009006C675
:10432600F074009006C7F0800C7400900105F074DC
:10433600199006C6F09000ECE06014741A9001061D
:10434600F074009006CAF074009006CBF0800C74EE
:1043560000900106F0741A9006CAF09000FEE06024
:1043660014742A900776F074009006C2F0740090D8
:1043760006C3F0800C7400900776F0742A9006C28B
:10438600F09000DEE0703274059006D6F074069068
:1043960006DAF074079006DEF074089006E2F07410
:1043A60000900772F07400900773F0740090077421
:1043B600F07400900775F0804874009006D6F0748B
:1043C600009006D7F074009006DAF074009006DBD1
:1043D600F074009006DEF074009006DFF074009032
:1043E60006E2F074009006E3F07405900772F0742C
:1043F60006900773F07407900774F07408900775B9
:10440600F09000CEE0D39402401A7415900766F03F
:104416007416900767F07417900768F07418900781
:1044260069F080277415900766F09000CEE0B4021C
:10443600087416900767F080067400900767F0749A
:1044460000900768F07400900769F0D2229000B2DD
:10445600E090006AF09000DEE090006BF09000D0F3
:10446600E090006DF09000C0E090006EF09000CEFD
:10447600E090006CF0900085E0900071F09000EB09
:10448600E090006FF09000ECE0900070F09000FE7D
:10449600E0900072F09000E8E0B4011790002074FC
:1044A6000FF0A374FFF0900022E4F0A3F0740290E2
:1044B60000E8F09000E8E0B40341900022E0FEA39B
:1044C600E0FF900020E0FCA3E0FD127105741012DD
:1044D60070BA7408120039EF9000E7F0EF700674B6
:1044E600FF9000E7F074009000E8F0900021E09063
:1044F600009EF0900020E090009FF0900079E09000
:104506000076F0900078E0900075F09000A7E0C388
:10451600941E50569000A7E0F404241E900077F0F5
:10452600900077E075F0B484FF7E008F749000777A
:10453600E075F0B484ADF07C008D75900075E0D325
:104546009575400D900075E0C39575900075F080E7
:104556000F900075E024B4C39575900075F005744E
:10456600900076E02574900076F0900076E090005A
:104576003AF090003AE00490003BF090003AE0D325
:104586009404400B90003AE0C3940490003AF090F3
:10459600003BE0D39404400B90003BE0C3940490AE
:1045A600003BF0C22690003AE0D39402400D900002
:1045B6003AE0C3940290003AF0D226C22790003B1C
:1045C600E0D39402400D90003BE0C3940290003B80
:1045D600F0D227755E01900079E0FE9000BFE0D32F
:1045E6009E5013900079E0FE9000BFE0F4042E0484
:1045F60090003CF08013900079E02404FE9000BF08
:10460600E0F4042E0490003CF090003CE0D39402C9
:10461600400F90003CE0C3940290003CF0D21D8015
:1046260002C21D90003CE0D39401400B90003CE098
:104636001490003DF0800990003CE00490003DF0AD
:1046460012019C22C293C294C291C292C287C290A6
:10465600E5B554EFF5B5E5B554DFF5B5C296C295A7
:10466600C2A0C297C2A2C2A1E5B554BFF5B5E5B5D1
:10467600547FF5B5E5B554FBF5B5C20C755F4690AC
:1046860000C2E07005756E028003756E03755500F5
:1046960075540090000874FFF0A374DCF0C211C2D8
:1046A6001474C8900036F074C8900038F075530042
:1046B600755200C204754700E570B41303757000A7
:1046C600756400900016E4F0A3F0757110C20FC275
:1046D60010C20375570075560090000AE4F0A3F067
:1046E60090000CE4F0A3F0C22975590075580090AB
:1046F6000084E075F032A4FFAEF090001EEEF0A349
:10470600EFF0900074E4F09008E2E4F0C225C21ADB
:10471600D21BC21CC21DC21E90000EE4F0A3F0C242
:1047260005C206900074E4F022755B00755A00AE6F
:104736005AAF5B741CC39F74019E500302482390BA
:104746006D6E120048E493645F6023906D6E1200F4
:1047560048E493647E6017906D6E120048E493649B
:1047660081600B906D6E120048E493B48403024896
:1047760003AE5AAF5B906D6E120048E493900078DA
:104786001270EB0FBF00010EE0FC906D6E12004838
:10479600ECFEE493FFEEC39F5026AE5AAF5B0FBF0D
:1047A60000010E906D6E120048AE5AAF5BE493FCAA
:1047B600906D6E120048E4939000781270EBECF066
:1047C600AE5AAF5B906D6E120048E493900078127B
:1047D60070EBE0FC906D70120048ECFCE493FDEC8D
:1047E600D39D4019906D70120048E493FC906D6E55
:1047F600120048E4939000781270EBECF0AE5AAFDA
:104806005B74022FFF50010E8E5A8F5B785B74012A
:1048160026F6500418E436F6400302473522755B47
:1048260000755A00AE5AAF5B7432BE00039F500348
:104836000248F1906E8B120048E493900078127053
:10484600EB0FBF00010EE0FC906E8B120048ECFEF1
:10485600E493FFEEC39F5026AE5AAF5B0FBF000135
:104866000E906E8B120048AE5AAF5BE493FC906ECE
:104876008B120048E4939000781270EBECF0AE5A7D
:10488600AF5B906E8B120048E4939000781270EB49
:10489600E0FC906E8D120048ECFCE493FDECD39D99
:1048A6004019906E8D120048E493FC906E8B1200B6
:1048B60048E4939000781270EBECF0AE5AAF5B745C
:1048C6002D6F4E7006755B33755A00AE5AAF5B742A
:1048D600022FFF50010E8E5A8F5B785B740126F60D
:1048E600500418E436F6400302482A22755B007528
:1048F6005A00AE5AAF5B7432BE00039F50030249A2
:10490600BF906EBE120048E4939000781270EB0FD1
:10491600BF00010EE0FC906EBE120048ECFEE49370
:10492600FFEEC39F5026AE5AAF5B0FBF00010E903D
:104936006EBE120048AE5AAF5BE493FC906EBE1298
:104946000048E4939000781270EBECF0AE5AAF5B3F
:10495600906EBE120048E4939000781270EBE0FC73
:10496600906EC0120048ECFCE493FDECD39D401918
:10497600906EC0120048E493FC906EBE120048E4AC
:10498600939000781270EBECF0AE5AAF5B742D6F1B
:104996004E7006755B33755A00AE5AAF5B74022FC4
:1049A600FF50010E8E5A8F5B785B740126F6500419
:1049B60018E436F640030248F822755B00755A0083
:1049C600AE5AAF5B7432BE00039F5003024A8D900D
:1049D6006EF1120048E4939000781270EB0FBF005E
:1049E600010EE0FC906EF1120048ECFEE493FFEE3F
:1049F600C39F5026AE5AAF5B0FBF00010E906EF1FB
:104A0600120048AE5AAF5BE493FC906EF112004878
:104A1600E4939000781270EBECF0AE5AAF5B906EB8
:104A2600F1120048E4939000781270EBE0FC906E6F
:104A3600F3120048ECFCE493FDECD39D4019906E14
:104A4600F3120048E493FC906EF1120048E4939050
:104A560000781270EBECF0AE5AAF5B742D6F4E70AF
:104A660006755B33755A00AE5AAF5B74022FFF5062
:104A7600010E8E5A8F5B785B740126F6500418E49B
:104A860036F640030249C62285F97485FA757E0119
:104A96007F00E5751270BAE5742FFF50010E8E5A2D
:104AA6008F5BAC5CAD5DEF2DFDEE3CFC8C5C8D5DF3
:104AB600D293D294D291D292E55DF5FBE55CF5FCFA
:104AC600E55DF5E9E55CF5EAE55DF5EBE55CF5EC5C
:104AD600E55DF5EDE55CF5EE2275A71085F97485C3
:104AE600FA757E017F00E5751270BAE5742FFF50E6
:104AF600010E8E5A8F5B7E017F769000FDE012706C
:104B0600BAAC5AAD5BED2FFFEC3EFE8E5C8F5DE5D9
:104B16005DF5FDE55CF5FE900066E4F075A70074B2
:104B260012900043F02285F97485FA757E017F00A4
:104B3600E5751270BAE5742FFF50010E8E5A8F5B21
:104B4600900010E0FCA3E0FDEF2DFDEE3CFC8C5C3C
:104B56008D5DE55DF5FDE55CF5FE22056522A2D8D5
:104B6600B34002C293A2D9B34002C294A2DAB340C0
:104B760002C291A2DBB34002C292A2DCB34030A2D1
:104B86009650067419900043F0A295500674199039
:104B96000043F0A2A050067419900043F0A297506B
:104BA600067419900043F0C296C295C2A0C29775CA
:104BB600D8402285A77375A710A2D8B34002C28732
:104BC600A2D9B34002C290A2DAB34006E5B554EFCB
:104BD600F5B5A2DBB34006E5B554DFF5B5A2DCB307
:104BE60040089000CCE0900066F075D8408573A729
:104BF6002290F800E4936406600280FE12009E751F
:104C0600A70075D80075D90475DA0975DB0975DC56
:104C16000975DD0975DE0975D84075A71075D800C8
:104C260075D90475DA0975DB0975DC0975DD097551
:104C3600DE0975D84075A7001200FB7509C875080E
:104C4600001205E475A70FE5FC900052F0E5FB9015
:104C56000053F0E5FA900054F0E5F9900055F07530
:104C6600A70090F800E493F52812070390088FE058
:104C7600D39403500790088FE0B40106740090089F
:104C86008FF090088FE09008E6F074019000C1F074
:104C960090088FE0906942F8282873802A8028754A
:104CA600A70F75F30F75A700A2A340067402900024
:104CB600C1F0801375A70F75F31775A700A2A4405E
:074CC6000674029000C1F02A
:0C694200024CA1024CA3024CA5024CBA6E
:104CCD009000C1E0B4022AC219120AAC740290001D
:104CDD00C1F090088FE090694EF8282873801080FD
:0F4CED000E74009000D0F0800674009000DDF08F
:0C694E00024CEA024CEC024CEE024CF64B
:104CFC008028D2191209C174019000C1F090088F5C
:104D0C00E090695AF82828738010800E7400900087
:0A4D1C00D0F0800674009000DDF076
:0C695A00024D14024D16024D18024D2093
:104D260090F807E49390005FF090005FE0440890ED
:104D3600005FF090005FE054FE90005FF012039D6C
:104D4600123EB790089CE0900164F090089DE090B8
:104D56000165F090089EE0900166F0900164E070B5
:104D66000C900165E07006900166E060028004C266
:104D7600238002D2239000B2E00490006AF012472A
:104D86002F90F802E493B405051248F2801290F8C9
:104D960002E493D39405400512482480031249C0C7
:104DA60074009000E8F0124003E5B54401F5B574CF
:104DB60006900045F07400900046F074019000479C
:104DC600F090F802E493900048F090F803E4939092
:104DD6000049F090F804E49390004AF074069000BD
:104DE6004BF0900048E0B40506740590004BF09037
:104DF6000048E0B40406740490004BF07430900050
:104E06004CF0740390004DF0740690004EF0740759
:104E160090004FF090F805E493900050F090F8065B
:104E2600E493900051F07400900059F074009000E3
:104E36005AF0740090005BF0740090005CF074000F
:104E460090005DF0740090005EF074FF900060F0DA
:104E5600A2B6B39208A2B3B39209A2A4B39220A2B7
:104E6600A3B39221900061E4F0757000743A900744
:104E760078F074FD900779F0900062E4F0756F01A8
:104E8600900043E4F09000C2E0B40106741A90006A
:104E960043F0C21F756400C20DD20EC203757200C4
:104EA600C222120586756000756C00756200756613
:104EB60032756700756800756900756A00756B0064
:104EC600900016E4F0A3F0756D00D2B2D2A4D2B071
:104ED600D2B1D2A3D2A7D2A6D2A5D2B77E017F00E5
:104EE60090009FE01270BA90009EE02FFF50010ED6
:104EF600900020EEF0A3EFF0EFD394FFEE940F4076
:104F060007900020E4F0A3F09000E7E0700674FF3D
:104F16009000E7F09000C2E07005756E02800375A0
:104F26006E037400900104F07400900107F07400A1
:104F3600900108F074299006BEF0740190076EF097
:104F4600740290076FF07403900770F07404900772
:104F560071F0740090076AF0740090076BF07400AB
:104F660090076CF0740090076DF0D29CE571D394B5
:104F76001040037571109006BFE0D3940C40067480
:104F8600009006BFF09006C3E0D3940C4006740070
:104F96009006C3F09006C7E0D3940C4006740090C8
:104FA60006C7F09006CBE0D3940C4006740090063A
:104FB600CBF09006CFE0D3940C400674009006CF59
:104FC600F09006D3E0D3940C400674009006D3F01C
:104FD6009006D7E0D3940C400674009006D7F09064
:104FE60006DBE0D3940C400674009006DBF09006D6
:104FF600DFE0D3940C400674009006DFF09006E3E1
:10500600E0D3940C400674009006E3F0D2EC75CF22
:1050160001A298B34005C298120C14E54E6006A290
:1050260099B3B340028005C2991210A3E54F6401FB
:105036006005E54FB4040280D5C28E7E087F00E588
:10504600651270BAE58D75F008A4FDACF0EF2DFD84
:10505600EE3CFCE58B75F02084FF7E00ED2FFFEC27
:105066003EFE8E548F55D28E9000A5E0605C900077
:10507600181270C8900018E0FCA3E0FD90001AE03A
:10508600FAA3E0FBEDB50342ECB5023EB217A2046B
:10509600B3401975E700A217B34008E5B54404F517
:1050A600B58006E5B554FBF5B575E71090001AE036
:1050B600FEA3E0FF90001CE0FCA3E0FDEF2DFDEE5B
:1050C6003CFC90001AECF0A3EDF09000B2E0600911
:1050D6009000B2E0C39403400302518D122FCEA27A
:1050E60004400890009CE0F546801BE560C395618E
:1050F6005005754600800F900089E0C39562500602
:105106009000AFE0F546E54675F002A4FFAEF090DC
:105116000884EEF0A3EFF075E700AC2FAD30EDD3C9
:105126009FEC9E402CE5B5547FF5B59006BFE07028
:1051360006E5B554F7F5B59000B2E0B40209900063
:10514600D0E0C3940240028006E5B54440F5B58040
:1051560033900061E0C39411502AE5B54480F5B55B
:105166009006BFE07006E5B54408F5B59000B2E0DC
:10517600B402099000D0E0C3940240028006E5B56F
:1051860054BFF5B575E7109000B2E0B4032A1230AB
:10519600E975E700AE2FAF30900884E0FCA3E0FD90
:1051A600EFD39DEE9C4008E5B54480F5B58006E555
:1051B600B5547FF5B575E710A2B3300901B3404188
:1051C600A2B3300901B34039A2B3300B01B3402476
:1051D600A2B6B3300701B34004B207800BA20CB3EA
:1051E60040067405900043F0A2B6B34002D21AA25C
:1051F6000BB39209A20BB330B301B34004A20B92D6
:1052060009A2B6300801B3500302576EA2B63008A1
:1052160001B3500302576EA2B6300A01B35003021F
:105226005681756F00A2B3B3300601B34004B206CF
:10523600800BA20CB340067405900043F0055FA2F4
:1052460005B3B35006A20CB3B34003025301E56E97
:10525600B4032EA229B34022E55FB40503756E019F
:10526600E55FC3940550069000437401F0E55FD3F3
:10527600940540067402900043F0755F01D22980C0
:105286005EE56EB40206756E01755F03E55FB403F5
:1052960005755F018049900043E07034E55FC39473
:1052A6000350069000437401F0E55FD39403400673
:1052B6007402900043F0E55FC394035002D21FE5E9
:1052C6005FD394034002D21FC296C295C2A0C29772
:1052D6009000C2E0B4010512464A8003755F01C220
:1052E6000574029008E2F0A21D921CD21BA2A2B382
:1052F6004002C219A21FB34002C21FE56EC3940347
:105306005006E55F640360028007B21CC21B755F2E
:1053160001E55FB4024F9000A5E06049900018E0F7
:10532600FEA3E0FF9000A5E08E048F05FF1270AA91
:1053360074018C068D0712003990001CEEF0A3EF65
:10534600F090001CE0F8A3E090001AC8F0A3C8F0A3
:10535600900018E4F0A3F0C21775E700E5B554FB1A
:10536600F5B575E710AE58AF59AC54AD55EF2DFDF8
:10537600EE3CFC8C588D59AE54AF55EFD39DEE9C48
:10538600401190000EE0FAA3E0FBEBC394E8EA9428
:10539600034002800690000E1270C8900008E55483
:1053A600F0A3E555F090000AE554F0A3E555F0AEFC
:1053B60054AF5574128E048F05FF1270AA8C568D49
:1053C60057C28E758D00758B007565007555017514
:1053D6005400D28E900008E0FEA3E0FFEF4E600B73
:1053E6007C7A7DAC126FA88E528F53AE52AF537437
:1053F60028BE00039F5010E5642FFF50010E740174
:105406001200398E528F538553649000C9E0A8521A
:10541600B8000DD395534008E553900042F080093B
:105426009000C9E014900042F0E56E6006755300E6
:105436007552009000C0E0B4040890003CE0655F3F
:105446006002800BA21CB34004D21E8002B21E90E2
:1054560000B2E06003122C84E570B413037570008B
:10546600A20D50030255D99000CEE0C39404500615
:10547600A20CB3B3400302552490007EE0B401733E
:10548600900100E0B40214121244900067E075F037
:10549600BCA4FFAEF08E5C8F5D8056E56875F00AA1
:1054A60084FF7E00900578120048E0F55B755A008F
:1054B600AE5AAF5B9000A3E01270BA74648E048F8C
:1054C60005FF1270AA8C5C8D5DE55D90003EF0AE26
:1054D6005AAF5B90007CE01270BA74648E048F053C
:1054E600FF1270AA74BC8C068D071270BA8E5C8F80
:1054F6005D801790007CE075F0BCA4FFAEF08E5C7A
:105506008F5D9000A3E090003EF0E562C394CC501E
:1055160006E55D455C70028003124A8ED20D90004E
:10552600CEE0B404069008E2E070030255D990007C
:105536007EE0B40173900100E0B4021412124490AC
:105546000067E075F0BCA4FFAEF08E5C8F5D805600
:10555600E56875F00A84FF7E00900578120048E041
:10556600F55B755A00AE5AAF5B9000A3E01270BAB5
:1055760074648E048F05FF1270AA8C5C8D5DE55DE8
:1055860090003EF0AE5AAF5B90007CE01270BA74A9
:10559600648E048F05FF1270AA74BC8C068D0712E8
:1055A60070BA8E5C8F5D801790007CE075F0BCA4AD
:1055B600FFAEF08E5C8F5D9000A3E090003EF0E5BC
:1055C60062C394CC5006E55D455C70028003124AC6
:1055D6008ED20DE56EB40106A20CB3B3400280185C
:1055E6009000CEE0B40405757103800975710090D2
:1055F60000447401F0756E00E56E705B9000C5E0C6
:10560600600D900066E0A852B800069553400280EF
:10561600299000C5E0B40208757103756D00800C11
:10562600C201756D00900016E4F0A3F0900066E0EC
:1056360060067409900043F0801D75710090003A71
:10564600E0B55F069000447401F090003BE0B55F62
:10565600067402900044F0A20AB39208A2B340086E
:10566600900074E004F08005900074E4F0900074FB
:10567600E0B40307D205900074E4F0A20AB330B692
:1056860001B3500302576E756F0175E700E5B54427
:1056960001F5B575E710740B900061F0A20A920847
:1056A600E55FD394474014D20CE55FD3944B400B8F
:1056B6007405900043F0D21F755F469000CDE0B4AC
:1056C6000107E56BC3944140028018E56BC394144F
:1056D60050087413900043F08006740E900043F057
:1056E60012464A90004BE0FE900048E0C39E4009F7
:1056F600900048E0D39408400974FB900043F012F0
:10570600464A900049E06015900049E0FE90004747
:10571600E06E600974FC900043F012464A90004A1D
:10572600E0601590004AE0FE90004CE06E6009745F
:10573600FE900043F012464A90088FE06006900003
:10574600FDE060028003120B97A2B340089000743C
:10575600E004F08005900074E4F0900074E0B40377
:1057660007D205900074E4F0A21FB34008C296C2A7
:1057760095C2A0C2979000FDE0600CAE52AF537484
:1057860014BE00059F40028037900085E090696650
:10579600F8282873802A8028A2A3B35005A221B333
:1057A60040028005124ADFD2218015A2A4B350051B
:1057B600A220B340028005124ADFD2208002800078
:1069660002579A02579C02579E0257B10257C40219
:0269760057C602
:1057C600A20FB3B3500890003CE0655F6003025A35
:1057D600C1A202B35006A201B3B34003025ABD9060
:1057E60000C0E0B404028003025A999008E2E0B4D3
:1057F60002028003025A8EA21EB3500302594712B8
:105806003CD8900111E0601F900014E0FEA3E0FF79
:10581600900109E01270BA74C88E048F05FF1270E9
:10582600AA8C5C8D5D800A900014E0F55CA3E0F51F
:105836005DAE5CAF5D745E1270BA74058E048F0542
:10584600FF1270AAAE5AAF5BED2FFFEC3EFE8E5CE8
:105856008F5D900034E0FCA3E0FDEF2DFDEE3CFCF7
:105866008C5C8D5D123D78A203B34068123D1790A3
:105876000111E0601F900014E0FEA3E0FF90010913
:10588600E01270BA74C88E048F05FF1270AA8C5C81
:105896008D5D800A900014E0F55CA3E0F55DAE5CDA
:1058A600AF5D745E1270BA74058E048F05FF1270B8
:1058B600AAAE5AAF5BED2FFFEC3EFE8E5C8F5D907D
:1058C6000034E0FCA3E0FDEF2DFDEE3CFC8C5C8D8E
:1058D6005D123DA49000DEE0B40263123D17900114
:1058E60011E0D39404401BAE2DAF2E90010DE012B3
:1058F60070BA74C88E048F05FF1270AA8C5C8D5D19
:105906008006852D5C852E5DAE5CAF5D745E127083
:10591600BA74058E048F05FF1270AAAE5AAF5BEDFE
:105926002FFFEC3EFE8E5C8F5D900034E0FCA3E022
:10593600FDEF2DFDEE3CFC8C5C8D5D123DA4025A04
:105946008C123CD8900111E0D39403401F900014B0
:10595600E0FEA3E0FF90010BE01270BA74C88E045B
:105966008F05FF1270AA8C5C8D5D800A900014E092
:10597600F55CA3E0F55DAE5CAF5D745E1270BA7463
:10598600058E048F05FF1270AAAE5AAF5BED2FFF8E
:10599600EC3EFE8E5C8F5D900034E0FCA3E0FDEFF4
:1059A6002DFDEE3CFC8C5C8D5D123D8EA203B3405A
:1059B6006B123D17900111E0D39403401F90001421
:1059C600E0FEA3E0FF90010BE01270BA74C88E04EB
:1059D6008F05FF1270AA8C5C8D5D800A900014E022
:1059E600F55CA3E0F55DAE5CAF5D745E1270BA74F3
:1059F600058E048F05FF1270AAAE5AAF5BED2FFF1E
:105A0600EC3EFE8E5C8F5D900034E0FCA3E0FDEF83
:105A16002DFDEE3CFC8C5C8D5D123DC69000DEE0FB
:105A2600B40263123D17900111E0D39406401BAEF9
:105A36002DAF2E90010FE01270BA74C88E048F0538
:105A4600FF1270AA8C5C8D5D8006852D5C852E5DAF
:105A5600AE5CAF5D745E1270BA74058E048F05FF7E
:105A66001270AAAE5AAF5BED2FFFEC3EFE8E5C8F36
:105A76005D900034E0FCA3E0FDEF2DFDEE3CFC8CD8
:105A86005C8D5D123DC68009123CD8123D78123DF0
:105A96008E8024123CD8123D78123D8EA203B3406C
:105AA60006123DA4123DC69000DEE0B40209123D86
:105AB60017123DA4123DC6C20FD210A210B3B350A6
:105AC6000890003DE0655F6003025DC2A202B3502C
:105AD60006A201B3B34003025DBE9000C0E0B40469
:105AE600028003025D9A9008E2E0B402028003029B
:105AF6005D8FA21EB35003025C48123CD890011180
:105B0600E0D39401401F900014E0FEA3E0FF900153
:105B16000AE01270BA74C88E048F05FF1270AA8C40
:105B26005C8D5D800A900014E0F55CA3E0F55DAE47
:105B36005CAF5D745E1270BA74058E048F05FF1239
:105B460070AAAE5AAF5BED2FFFEC3EFE8E5C8F5D0A
:105B5600900034E0FCA3E0FDEF2DFDEE3CFC8C5CF8
:105B66008D5D123D83A203B3406B123D1790011168
:105B7600E0D39401401F900014E0FEA3E0FF9001E3
:105B86000AE01270BA74C88E048F05FF1270AA8CD0
:105B96005C8D5D800A900014E0F55CA3E0F55DAED7
:105BA6005CAF5D745E1270BA74058E048F05FF12C9
:105BB60070AAAE5AAF5BED2FFFEC3EFE8E5C8F5D9A
:105BC600900034E0FCA3E0FDEF2DFDEE3CFC8C5C88
:105BD6008D5D123DB59000DEE0B40263123D179074
:105BE6000111E0D39405401BAE2DAF2E90010EE0BF
:105BF6001270BA74C88E048F05FF1270AA8C5C8D61
:105C06005D8006852D5C852E5DAE5CAF5D745E1293
:105C160070BA74058E048F05FF1270AAAE5AAF5B78
:105C2600ED2FFFEC3EFE8E5C8F5D900034E0FCA312
:105C3600E0FDEF2DFDEE3CFC8C5C8D5D123DB5026A
:105C46005D8D123CD8900111E0D39403401F900063
:105C560014E0FEA3E0FF90010CE01270BA74C88E47
:105C6600048F05FF1270AA8C5C8D5D800A9000146B
:105C7600E0F55CA3E0F55DAE5CAF5D745E1270BAF4
:105C860074058E048F05FF1270AAAE5AAF5BED2F16
:105C9600FFEC3EFE8E5C8F5D900034E0FCA3E0FDE1
:105CA600EF2DFDEE3CFC8C5C8D5D123D99A203B39D
:105CB600406B123D17900111E0D39403401F9000F2
:105CC60014E0FEA3E0FF90010CE01270BA74C88ED7
:105CD600048F05FF1270AA8C5C8D5D800A900014FB
:105CE600E0F55CA3E0F55DAE5CAF5D745E1270BA84
:105CF60074058E048F05FF1270AAAE5AAF5BED2FA6
:105D0600FFEC3EFE8E5C8F5D900034E0FCA3E0FD70
:105D1600EF2DFDEE3CFC8C5C8D5D123DDB9000DED4
:105D2600E0B40263123D17900111E0D39407401BC3
:105D3600AE2DAF2E900110E01270BA74C88E048F8B
:105D460005FF1270AA8C5C8D5D8006852D5C852E04
:105D56005DAE5CAF5D745E1270BA74058E048F051D
:105D6600FF1270AAAE5AAF5BED2FFFEC3EFE8E5CC3
:105D76008F5D900034E0FCA3E0FDEF2DFDEE3CFCD2
:105D86008C5C8D5D123DDB8009123CD8123D83127E
:105D96003D998024123CD8123D83123D99A203B34B
:105DA6004006123DB5123DDB9000DEE0B40209125A
:105DB6003D17123DB5123DDBD20FC210E571906959
:095DC60078F82828739000E5E04C
:03697800025DCBF2
:105DCF009069E7F82828731225CF80121225CF800B
:0E5DDF000D1226598008122705800312270591
:0F69E700025DD6025DDB025DE0025DE5025DEA66
:105DED007571010261B412283112294875710202D0
:105DFD0061B4122CC8A204B340139000CAE075F030
:105E0D001DA4FFAEF0900010EEF0A3EFF090087817
:105E1D00E0FEA3E0FF740A1270BA90000AE0FCA342
:105E2D00E0FD74098F02FF1270AA8D078C038E049A
:105E3D008A058B06126FA890087CEEF0A3EFF09008
:105E4D0000CEE0B401087478BE00059F4002800DBD
:105E5D00747890087CF8E4F0E8A3F0801B90087C3F
:105E6D00E0FEA3E0FF74F0BE00039F500B74F090B2
:105E7D00087CF8E4F0E8A3F0E5377003753701907E
:105E8D00087CE0FEA3E0FFE5372FFF50010E9008E0
:105E9D007CEEF0A3EFF0757103A230401590004435
:015EAD00E014
:06697B00025DF3025DFF66
:105EAE009069F6F8282873800875710A8003757159
:015EBE000BD8
:0969F600025EB5025EB7025EBC50
:105EBF000261B49006BFE060077401F508122DF679
:105ECF00A232B3401675E700900776E0B42A06E5D4
:105EDF00B54402F5B575E710025F8B9000B3E0D3C0
:105EEF0094024045900087E02403A852B80004951F
:105EFF00535009900089E0D395625002800ED20270
:105F0F00A22840067408900043F0D228900087E042
:105F1F00A852B80005D39553500B900089E0240385
:105F2F00C395625002C2028053900087E02403A8F9
:105F3F0052B8000495535010E560C3956150099015
:105F4F000089E0D395625002800ED202A22840064B
:105F5F007408900043F0D228900087E0A852B80050
:105F6F0005D395535014E561240FC39560400B90F2
:105F7F000089E02403C395625002C202A2024002CC
:105F8F00C228A232B35005A202B34002801375E7B4
:105F9F0000900776E0B42A06E5B554FDF5B575E730
:105FAF00109000CDE07007E56BC39414400280029F
:105FBF00D2029000C2E0B40102D202A202400575E3
:105FCF007104800A757110900016E4F0A3F002615D
:055FDF00B49000B3E0E6
:06698100025EC2025FE0AD
:105FE4009069FFF828287312135A801212135A80EA
:0E5FF4000D12150D80081215C480031215C47D
:0F69FF00025FEB025FF0025FF5025FFA025FFFDB
:106002009006C3E060077402F508122DF67571055B
:106012000261B412171D7571069006C7E06007741D
:1060220003F508122DF69006CBE060077404F5081C
:10603200122DF60261B490003EE06006A204B3B3F2
:106042004002800DE55FD39401500690003EE014BB
:10605200F01219A67571079006CFE060077405F576
:1060620008122DF69006D3E060077406F508122D8B
:10607200F60261B4900100E0B402031212CB121EC8
:106082000E7571089006D7E060077407F508122DA7
:10609200F69006DBE060077408F508122DF602613F
:1060A200B4121EF07571090261B41222C8A20FB3B4
:1060B2005005A210B340028004D20FD210757110A5
:1060C2009006DFE060077409F508122DF69006E3EA
:1060D200E06007740AF508122DF60261B4900037E9
:1060E200E0C39446500AC296C2A07446900037F0AC
:1060F20085375B755A0090003AE0F574123F95E5DA
:106102005D900037F0900004E55AF0A3E55BF0C221
:106112001290087CE0F55AA3E0F55B90003AE0F5B6
:1061220074123F95E55D900036F0900000E55AF05C
:10613200A3E55BF0A2009213C21175710380739004
:106142000039E0C3944650139000CEE0B40102C27D
:1061520096C295C2977446900039F085375B755A9E
:106162000090003BE0F574123F95E55D900039F038
:10617200900006E55AF0A3E55BF0C21590087CE0BA
:10618200F55AA3E0F55B90003BE0F574123F95E50C
:106192005D900038F0900002E55AF0A3E55BF0A2B2
:1061A200009216C214757103800880068004800272
:0261B20080006B
:106987000260150260380260760260A30260AC0202
:1069970060DF0261410261AC0261AE0261B0026177
:0469A700B20261B423
:1061B400900036E0B55F02800302628AA211406B50
:1061C400900000E0FEA3E0FFEF4E605DAC52AD53E3
:1061D400740ABC0033D39D402FAA56AB5774058A6A
:1061E400048B05FF1270AA8D068C07900000E0FC5A
:1061F400A3E0FDCFCECF120003740112003990004A
:1062040000EEF0A3EFF08021AE56AF57900000E00F
:10621400FCA3E0FD120003740A8E048F05FF1270C4
:10622400AA900000ECF0A3EDF0D211AE54AF55905B
:106234000000E0FCA3E0FDEFC39DEE9C4048124B40
:106244002C9000CEE09069ABF82828738030D29669
:10625400802CD2968028D296D2A08022A2134010FD
:10626400A226301B01B34004D2A08002D296800E35
:0E627400A226301B01B34004D2968002D2A0B5
:0F69AB0002625002625202625602625A02626037
:10628200C21174C8900036F0A211B3B35007900047
:1062920036E0B55F028048124B2C9000CEE0906948
:1062A200BAF82828738030D296802CD2968028D2D1
:1062B20096D2A08022A2134010A226301B01B34026
:1062C20004D2A08002D296800EA226301B01B340D7
:0762D20004D2968002D2A065
:0F69BA000262A70262A90262AD0262B10262B775
:1062D90074C8900036F0C211900037E0B55F0280B3
:1062E9000302637BA212406B900004E0FEA3E0FF6F
:1062F900EF4E605DAC52AD53740ABC0033D39D4080
:106309002FAA56AB5774058A048B05FF1270AA8D04
:10631900068C07900004E0FCA3E0FDCFCECF12006D
:10632900037401120039900004EEF0A3EFF080210C
:10633900AE56AF57900004E0FCA3E0FD12000374D1
:106349000A8E048F05FF1270AA900004ECF0A3EDE9
:10635900F0D212AE54AF55900004E0FCA3E0FDEF7B
:10636900C39DEE9C400CC296C2A07446900037F0C3
:10637900C212A212B3B35007900037E0B55F028092
:106389000CC296C2A07446900037F0C21290003831
:10639900E0B55F02800302646CA214406B900002B6
:1063A900E0FEA3E0FFEF4E605DAC52AD53740ABC52
:1063B9000033D39D402FAA56AB5774058A048B0529
:1063C900FF1270AA8D068C07900002E0FCA3E0FD85
:1063D900CFCECF1200037401120039900002EEF003
:1063E900A3EFF08021AE56AF57900002E0FCA3E086
:1063F900FD120003740A8E048F05FF1270AA900023
:1064090002ECF0A3EDF0D214AE54AF55900002E0C7
:10641900FCA3E0FDEFC39DEE9C4048124B2C90007D
:10642900CEE09069C9F82828738030D296802CD2A2
:10643900958028D295D2978022A2164010A22730A3
:106449001B01B34004D2978002D295800EA2273057
:0B6459001B01B34004D2958002D297D3
:0F69C90002643202643402643802643C026442A5
:10646400C21474C8900038F0A214B3B3500790005B
:1064740038E0B55F028048124B2C9000CEE0906962
:10648400D8F82828738030D296802CD2958028D2D0
:1064940095D2978022A2164010A227301B01B34048
:1064A40004D2978002D295800EA227301B01B340FC
:0764B40004D2958002D2978B
:0F69D80002648902648B02648F026493026499E3
:1064BB0074C8900038F0C214900039E0B55F0280C8
:1064CB0003026566A215406B900006E0FEA3E0FF99
:1064DB00EF4E605DAC52AD53740ABC0033D39D409C
:1064EB002FAA56AB5774058A048B05FF1270AA8D21
:1064FB00068C07900006E0FCA3E0FDCFCECF120088
:10650B00037401120039900006EEF0A3EFF0802126
:10651B00AE56AF57900006E0FCA3E0FD12000374EB
:10652B000A8E048F05FF1270AA900006ECF0A3ED03
:10653B00F0D215AE54AF55900006E0FCA3E0FDEF92
:10654B00C39DEE9C40159000CEE0B40102C296C2F2
:10655B0095C2977446900039F0C215A215B3B3508B
:10656B0007900039E0B55F0280159000CEE0B401D2
:10657B0002C296C295C2977446900039F0C215902C
:10658B0000D0E0B4020280030266BE900063E0D349
:10659B0095675064900063E0F4042567FE9000D388
:1065AB00E08E00F5F0E884FF7E008F74EFC394104B
:1065BB00500CEF8574F0A4FDACF08D7480037574F2
:1065CB00FF900063E0D39574400B900063E0C3959C
:1065DB0074F57280037572009000EEE0D3957240F3
:1065EB00069000EEE0F5729000EFE0C39572500656
:1065FB009000EFE0F5728071900063E0C39567FE49
:10660B009000D3E08E00F5F0E884FF7E008F74EFEE
:10661B00C39410500CEF8574F0A4FDACF08D748016
:10662B00037574FF85745B755A00900063E0255BFE
:10663B00FFAE5A50010E8E5A8F5B74FFBE0009D30A
:10664B009F4005855B7280037572FF9000EEE0D36F
:10665B00957240069000EEE0F5729000EFE0C39566
:10666B007250069000EFE0F572A204B3B3500D9098
:10667B000064E0FE9000DBE0D39E500280147407B0
:10668B00900043F075E700E5B554BFF5B575E7101D
:10669B00802175A71075E700E5CDC395724008E51D
:1066AB00B554BFF5B58006E5B54440F5B575E710B3
:1066BB0075A7009000EBE0604E9000F5E0A852B893
:1066CB000004955350179000F4E0A852B8000ED375
:1066DB00955340099000F6E0D39562400280157502
:1066EB00A710E5CDC394BF4004C2A28002D2A2750D
:1066FB00A700801375A710E5CDC394404004C2A238
:10670B008002D2A275A7009000ECE0604E9000F8DA
:10671B00E0A852B80004955350179000F7E0A85228
:10672B00B8000ED3955340099000F9E0D395624021
:10673B0002801575A710E5CDC394BF4004C2A1809C
:10674B0002D2A175A700801375A710E5CDC39440A5
:10675B004004C2A18002D2A175A700E570C39413B7
:10676B00501DE57075F00284AFF07E00EF4E7005A2
:10677B00123290800AA2EDB34005C2ED123290AEF8
:10678B0054AF5574B8C39F74889E400C900062E060
:10679B00C3945A400302691EA20CB3400912464A25
:1067AB007406900043F0A20EB3500EE562D39433FF
:1067BB004007E562C394CC40028041900100E0B4F5
:1067CB000214121244900067E075F05EA4FFAEF065
:1067DB008E5C8F5D800F90007CE075F05EA4FFAE49
:1067EB00F08E5C8F5DE55D455C6011E5B54401F5B0
:1067FB00B5740B900061F0124A8ED20E900062E0DD
:10680B00D394014007E562C3941A40028002C20E82
:10681B009006BFE060077401F508122DF69006C3D1
:10682B00E060077402F508122DF69006C7E06007CA
:10683B007403F508122DF69006CBE060077404F58F
:10684B0008122DF69006CFE060077405F508122D9F
:10685B00F69006D3E060077406F508122DF6900645
:10686B00D7E060077407F508122DF69006DBE060A1
:10687B00077408F508122DF69006DFE0600774091F
:10688B00F508122DF69006E3E06007740AF508127E
:10689B002DF6900062E0C3945A5010E570B41309C2
:1068AB00900062E004F0757000803FE570B4130354
:1068BB00757000C28E758D00758B007565007555F2
:1068CB0001755400D28E900061E0C3941150089072
:1068DB000061E004F080067411900061F09000619B
:1068EB00E0B41106E5B554FEF5B5900062E0D39423
:1068FB00014007E56BC3944140028006740E900083
:10690B0043F090088FE060069000FDE0600280038A
:06691B00120B970250145C
:106A0E000000010001400160018001A001C001E011
:106A1E0002000300039603B603D603F40400050038
:106A2E000512052405360548055A056C057E0590A8
:106A3E0005A805C005DE0600061406280646066EE5
:106A4E0006AE05CF06EE00FF013F015F017F019FFD
:106A5E0001BF01DF01FF02FF039503B503D503F369
:106A6E0003FF04FF05110523053505470559056B81
:106A7E00057D058F05A705BF05CE05F10613062773
:106A8E000645066D06AD06ED05DD06FF0FAA0FA540
:106A9E000F9F0F9A0F940F8D0F870F800F780F7126
:106AAE000F680F600F570F4E0F450F3B0F300F251E
:106ABE000F1A0F0E0F020EF50EE80EDB0ECC0EBEE9
:106ACE000EAE0E9F0E8E0E7D0E6C0E5A0E470E34AF
:106ADE000E200E0C0DF70DE20DCB0DB50D9D0D8597
:106AEE000D6D0D540D3A0D200D050CE90CCE0CB1AB
:106AFE000C940C760C580C3A0C1B0BFB0BDB0BBBE3
:106B0E000B9A0B790B570B350B130AF10ACE0AAB06
:106B1E000A870A640A400A1C09F809D409B0098CCC
:106B2E0009670943091F08FB08D608B2088E086AD0
:106B3E000846082307FF07DC07B9079607730751B6
:106B4E00072F070D06EC06CA06AA0689066906492E
:106B5E00062A060A05EC05CD05B005920575055801
:106B6E00053C0520050504EA04CF04B5049C048207
:106B7E000469045104390422040B03F403DE03C830
:106B8E0003B2039D038903750361034D033B032881
:106B9E000316030402F202E102D102C002B002A007
:106BAE00029102820273026502570249023C022FD1
:106BBE0002220216020901FD01F201E601DB01D0FB
:106BCE0001C601BB01B101A7019D0194018B018298
:106BDE0001790170016801600158015001480141BD
:106BEE0001390132012B0125011E01180111010B82
:106BFE00010500FF00FA0FA60FA00F990F920F8B41
:106C0E000F840F7C0F740F6B0F620F580F4E0F43D4
:106C1E000F380F2C0F1F0F120F050EF70EE80ED8A0
:106C2E000EC80EB70EA50E930E800E6C0E580E42A9
:106C3E000E2C0E150DFD0DE40DCB0DB10D950D7930
:106C4E000D5D0D3F0D200D010CE10CC00C9E0C7C5A
:106C5E000C590C350C100BEA0BC40B9E0B760B4F1C
:106C6E000B260AFD0AD40AAA0A800A550A2A09FF27
:106C7E0009D409A8097C0950092508F908CD08A1ED
:106C8E000875084A081E07F307C8079D07730749CA
:106C9E00072006F706CE06A6067E06570630060A1B
:106CAE0005E405BF059B057705540532051004EF75
:106CBE0004CE04AE048F047104530435041903FD8D
:106CCE0003E203C703AD0394037B0363034B033457
:106CDE00031E030802F302DE02CA02B602A30291E9
:106CEE00027F026D025C024C023C022C021D020E5F
:106CFE00020001F201E401D701CA01BE01B101A6F1
:106D0E00019A018F0185017A01700166015D0153BF
:106D1E00014A0141013901310129012101190112F3
:106D2E00010B010400FD00F700F000EA00E400DEB4
:106D3E0000D900D300CE00C900C400BF00BA00B510
:106D4E0000B100AD00A800A400A0009C0099009521
:106D5E000091008E008A008700840081007E007BF7
:10009E0075B50075840175A70075FFA075EF069004
:1000AE00003FE4F075C91075A70F75A1C775A700BD
:1000BE0075D90075CE0C75A70F75F1FE75F2FF752B
:1000CE00F30775F47875A4BA75A5FF75A60775AE16
:1000DE000075AFFF75D48175D5FF75D6FF75D7FF47
:1000EE0075A70075A20175A14775F8092275E60876
:1000FE0075E71075BC0175BE0475BD6C75BE0775D0
:10010E00BDA075BE0875BD0175BC0075BB1875BC6C
:10011E002075BA0875E88075D11375A70F75E105BE
:10012E0075E20075C74012464A7597007597807440
:10013E000A12709A7597C0E5975420700280F87570
:10014E008F0275A700D2AF75980075A90C75A70F11
:10015E0075AB4375ADFB75AC1E75A71075C91875DB
:10016E00CA0075CB0075C80475A700758912758E07
:10017E0004758C00758A00C2A9D28C758D00758BA2
:10018E0000D2ABD28E75B62075D944C2992290009A
:10019E007AE090088EF0900085E090088FF0900045
:1001AE0086E0900890F09000A5E0900891F0900005
:1001BE00B2E0900892F09000C0E0900893F09000AA
:1001CE00CEE0900894F09000D0E0900895F090006A
:1001DE00DEE0900896F09000EBE0900897F090002B
:1001EE00ECE0900898F09000FEE0900899F09001F5
:1001FE0016E090089BF0900164E090089CF090014E
:10020E0065E090089DF0900166E090089EF09000E9
:10021E00FDE090089FF09000E7E09008A0F09000BD
:10022E009EE09008A1F090009FE09008A2F0900050
:10023E0099E09008A3F090009AE09008A4F0900145
:10024E0003E09008A5F0900104E09008A6F090015C
:10025E0005E09008A7F0900106E09008A8F0900144
:10026E0007E09008A9F09006BEE09008AAF090066C
:10027E00C2E09008ABF09006C6E09008ACF0900695
:10028E00CAE09008ADF09006CEE09008AEF0900671
:10029E00D2E09008AFF09006D6E09008B0F090064D
:1002AE00DAE09008B1F09006DEE09008B2F0900629
:1002BE00E2E09008B3F0900766E09008B4F0900783
:1002CE0067E09008B5F0900768E09008B6F09007E8
:1002DE0069E09008B7F090076AE09008B8F09007D0
:1002EE006BE09008B9F090076CE09008BAF09007B8
:1002FE006DE09008BBF090076EE09008BCF09007A0
:10030E006FE09008BDF0900770E09008BEF0900787
:10031E0071E09008BFF0900772E09008C0F090076F
:10032E0073E09008C1F0900774E09008C2F0900757
:10033E0075E09008C3F0900776E09008C4F0900145
:10034E0008E09008C5F0900109E09008C6F0900111
:10035E000AE09008C7F090010BE09008C8F09001F9
:10036E000CE09008C9F090010DE09008CAF09001E1
:10037E000EE09008CBF090010FE09008CCF09001C9
:10038E0010E09008CDF0900111E09008CEF0229090
:10039E00088EE090007AF090088FE0900085F09043
:1003AE000890E0900086F0900891E09000A5F09003
:1003BE000892E09000B2F0900893E09000C0F090A8
:1003CE000894E09000CEF0900895E09000D0F09068
:1003DE000896E09000DEF0900897E09000EBF09029
:1003EE000898E09000ECF0900899E09000FEF090F4
:1003FE00089BE0900116F090089FE09000FDF090B1
:10040E0008A0E09000E7F09008A1E090009EF09028
:10041E0008A2E090009FF09008A3E0900099F09061
:10042E0008A4E090009AF09008A5E0900103F090E7
:10043E0008A6E0900104F09008A7E0900105F09066
:10044E0008A8E0900106F09008A9E0900107F0904E
:10045E0008AAE09006BEF09008ABE09006C2F090BD
:10046E0008ACE09006C6F09008ADE09006CAF09099
:10047E0008AEE09006CEF09008AFE09006D2F09075
:10048E0008B0E09006D6F09008B1E09006DAF09051
:10049E0008B2E09006DEF09008B3E09006E2F0902D
:1004AE0008B4E0900766F09008B5E0900767F0900A
:1004BE0008B6E0900768F09008B7E0900769F090F2
:1004CE0008B8E090076AF09008B9E090076BF090DA
:1004DE0008BAE090076CF09008BBE090076DF090C2
:1004EE0008BCE090076EF09008BDE090076FF090AA
:1004FE0008BEE0900770F09008BFE0900771F09092
:10050E0008C0E0900772F09008C1E0900773F09079
:10051E0008C2E0900774F09008C3E0900775F09061
:10052E0008C4E0900776F09008C5E0900108F090BE
:10053E0008C6E0900109F09008C7E090010AF0901B
:10054E0008C8E090010BF09008C9E090010CF09003
:10055E0008CAE090010DF09008CBE090010EF090EB
:10056E0008CCE090010FF09008CDE0900110F090D3
:10057E0008CEE0900111F022754800900886E4F054
:10058E00A3F0753200753100754E00754F00C22C08
:10059E00D22D90088FE06002D22274FE900888F867
:1005AE00E4F0E8A3F074FE90088CF8E4F0E8A3F011
:1005BE0074FE90088AF8E4F0E8A3F0745A9008E00C
:1005CE00F0745A9008E1F0D22EC22AC230C22FC265
:1005DE002BC232C23822750B00750A00AE0AAF0B61
:1005EE00AC08AD09EDC39FEC9E401674FF12709AD5
:1005FE0075CF01780B740126F6500418E436F650C8
:10060E00DB22C2AF75D904758F0375B7A575B7F127
:10061E0090F800E4F0758F0175B7A575B7F1E52870
:10062E0090F800F075B7A575B7F190F801E4F07584
:10063E00B7A575B7F19008D4E090F802F075B7A59C
:10064E0075B7F19008D8E090F803F075B7A575B7B7
:10065E00F19008D5E090F804F075B7A575B7F19054
:10066E0008D6E090F805F075B7A575B7F19008D7E4
:10067E00E090F806F075B7A575B7F19008D9E0903F
:10068E00F807F0758F0075D944D2AF2290003FE085
:10069E00B4AB61C2AF75D90475B62275F522758FEC
:1006AE000375B7A575B7F1740090F600F0758F015C
:1006BE00755B00755A00AE5AAF5B7445BE00279F3E
:1006CE00402475B7A575B7F190088E120048E0FC6E
:1006DE0090F600120048ECF0785B740126F6500498
:1006EE0018E436F650D0758F0075F51175B6207575
:1006FE00D944D2AF22C2AF75F52275D904755B000D
:10070E00755A00AE5AAF5B7445BE00229F401F90D3
:10071E00F600120048E493FC90088E120048ECF0AC
:10072E00785B740126F6500418E436F650D575D968
:10073E004475F511D2AF2290003FE0B4AA028003B7
:10074E00020882C2AF75D90475B62275F522758F6F
:10075E000375B7A575B7F1740090F400F075B7A5E1
:10076E0075B7F1740090F200F075B7A575B7F17416
:10077E000090F000F075B7A575B7F1740090EE001B
:10078E00F0758F01755B00755A00AE5AAF5B74FF42
:10079E00C39F74019E402475B7A575B7F19000787C
:1007AE00120048E0FC90F400120048ECF0785B7404
:1007BE000126F6500418E436F650CF755B00755AD4
:1007CE0000AE5AAF5B74FFC39F74019E402475B791
:1007DE00A575B7F1900278120048E0FC90F2001275
:1007EE000048ECF0785B740126F6500418E436F6F7
:1007FE0050CF755B00755A00AE5AAF5B74FFC39F46
:10080E0074019E402475B7A575B7F1900478120057
:10081E0048E0FC90F000120048ECF0785B74012682
:10082E00F6500418E436F650CF755B00755A00AEDC
:10083E005AAF5B74FFC39F74019E402475B7A575B4
:10084E00B7F1900678120048E0FC90EE00120048D6
:10085E00ECF0785B740126F6500418E436F650CFAF
:10086E00758F0075F51175B62075D944D2AF743AEF
:10087E00900778F02290003FE0B4AA0280030209AC
:10088E00C0C2AF75D90475B62275F522758F037582
:10089E00B7A575B7F1740090EC00F075B7A575B7F4
:1008AE00F1740090EA00F075B7A575B7F174009079
:1008BE00E800F075B7A575B7F1740090E600F07515
:1008CE008F01755B00755A00AE5AAF5B74FFC39F04
:1008DE0074019E402475B7A575B7F190007812008B
:1008EE0048E0FC90EC00120048ECF0785B740126B6
:1008FE00F6500418E436F650CF755B00755A00AE0C
:10090E005AAF5B74FFC39F74019E402475B7A575E3
:10091E00B7F1900278120048E0FC90EA001200480D
:10092E00ECF0785B740126F6500418E436F650CFDE
:10093E00755B00755A00AE5AAF5B74FFC39F7401AE
:10094E009E402475B7A575B7F1900478120048E063
:10095E00FC90E800120048ECF0785B740126F6502B
:10096E000418E436F650CF755B00755A00AE5AAFD8
:10097E005B74FFC39F74019E402475B7A575B7F1D4
:10098E00900678120048E0FC90E600120048ECF069
:10099E00785B740126F6500418E436F650CF758F46
:1009AE000075F51175B62075D944D2AF743A90071B
:1009BE0078F022C2AF75D90475F522755B00755AB1
:1009CE0000AE5AAF5B74FFC39F74019E401F90F43C
:1009DE0000120048E493FC900078120048ECF07886
:1009EE005B740126F6500418E436F650D4755B009D
:1009FE00755A00AE5AAF5B74FFC39F74019E401FC1
:100A0E0090F200120048E493FC900278120048EC39
:100A1E00F0785B740126F6500418E436F650D4755F
:100A2E005B00755A00AE5AAF5B74FFC39F74019E94
:100A3E00401F90F000120048E493FC9004781200DE
:100A4E0048ECF0785B740126F6500418E436F65044
:100A5E00D4755B00755A00AE5AAF5B74FFC39F74BA
:100A6E00019E401F90EE00120048E493FC90067821
:100A7E00120048ECF0785B740126F6500418E43648
:100A8E00F650D475F51175D944D2AF74019000C1EA
:100A9E00F0743A900778F09008E77401F022C2AF34
:100AAE0075D90475F522755B00755A00AE5AAF5BA9
:100ABE0074FFC39F74019E401F90EC00120048E427
:100ACE0093FC900078120048ECF0785B740126F6E7
:100ADE00500418E436F650D4755B00755A00AE5AC1
:100AEE00AF5B74FFC39F74019E401F90EA0012001B
:100AFE0048E493FC900278120048ECF0785B7401A5
:100B0E0026F6500418E436F650D4755B00755A007C
:100B1E00AE5AAF5B74FFC39F74019E401F90E800F6
:100B2E00120048E493FC900478120048ECF0785BD5
:100B3E00740126F6500418E436F650D4755B007531
:100B4E005A00AE5AAF5B74FFC39F74019E401F9054
:100B5E00E600120048E493FC900678120048ECF090
:100B6E00785B740126F6500418E436F650D475F509
:100B7E001175D944D2AF74029000C1F0743A900747
:100B8E0078F074029008E7F02274019000C1F090A2
:100B9E00088FE0903C1EF828287380188016A2A3B8
:100BAE00400674029000C1F0800AA2A440067402AE
:040BBE009000C1F0F2
:0C3C1E00020BA8020BAA020BAC020BB8B0
:100BC2009000C1E0B40105A236B34002801AD236C9
:100BD20012464A1209C174019000C1F012039D121B
:100BE2003EB7741B900043F09000C1E0B40206A22D
:100BF20036B3B34002801AC23612464A120AAC74A5
:100C0200029000C1F012039D123EB7741B90004384
:100C1200F022E54F64046006E59964FF60028031CA
:100C2200A22C4004D22C8027E54F600874E6254FA1
:100C3200900043F0E54E600874F0254E900043F0BA
:100C4200E54FB4010280FE754F00754E00C22C8044
:100C520002C22CE54F903C2AF8282873754F00E514
:100C620099B4FF03754E01E599B4FE03754E02E592
:100C720099B4FD03754E03E599B4FC03754E04E582
:100C820099B4FA03754E05E599B4FB06754F011246
:100C9200464AE599B4F906754F0412464AE599B4F5
:100CA200F73312464AC29C74AB90003FF012069A88
:100CB20074AA90003FF09008E7E0B40105120745DE
:100CC200800312088390003FE4F0D29C754F0075B8
:100CD2004E007599F7E599D394E54007E599C394D9
:100CE200F040028016859950754F027E017F00E523
:100CF20050C394E61270BA8E338F34900886E4F0B3
:100D0200A3F0E599D394C24007E599C394E6400263
:100D12008028859950754F0374E5C39550F5347555
:100D22003300AE33AF34906A0E127089E493F874D4
:100D32000193900886C8F0A3C8F0D2990210A2903D
:100D4200089BE0700AA223B35005A224B34002809C
:100D52005C900886E0FEA3E0FF74FFBE00039F5094
:100D620009EFC39446EE9406402B900886E0FEA35A
:100D7200E0FFEFD3946DEE94064009EFC394EEEEDC
:100D820094064011900886E0FEA3E0FFEFD394FFA3
:100D9200EE94064013900886E0FEA3E0FF900078F0
:100DA200120048E599F080038599758011900886B4
:100DB200E0FEA3E0FF900078120048E599F0900869
:100DC200861270C8900886E0FEA3E0FFEFB4010629
:100DD200EEB407028003020E9B900778E0B43C0257
:100DE2008003020E9BA223B35005A224B3400280CB
:100DF20055C29C12039D900085E09008E6F01240D7
:100E020003900164E090089CF0900165E090089DD9
:100E1200F0900166E090089EF074AB90003FF012F3
:100E2200069A74AA90003FF09008E7E0B401051218
:100E3200074580031208839008E7E09000C1F09014
:100E4200003FE4F08048C29C12019C740090089C10
:100E5200F0740090089DF0740090089EF090008558
:100E6200E09008E6F012400374AB90003FF01206E7
:100E72009A74AA90003FF0120745120883D29C751B
:100E820099FB7464F5097508001205E480FED29C92
:100E9200754F00754E007599FB0210A2900886E00E
:100EA200FEA3E0FFEF4E700685993275310090087F
:100EB20086E0FEA3E0FF74016F4E701BAC31AD32D1
:100EC200AA33AB34ED2BFBEC3AFA8A068B0790007F
:100ED20078120048E599F09008861270C89008864A
:100EE200E0FEA3E0FF74026F4E7021AC31AD3274AC
:100EF200566D4C7006E55064E66002800312464A65
:100F0200124003855099754F00754E000210A29051
:100F12000886E0FEA3E0FF900078120048E599F011
:100F22009008861270C8900886E0FEA3E0FFAC33FA
:100F3200AD348F028E038C068D07906A541270892D
:100F4200E493F9740193FEEAD39EEB99400985502C
:100F520099754F00754E000210A2900886E0FEA31C
:100F6200E0FF900078120048E599F0900886127030
:100F7200C8900886E0FEA3E0FFEFB40006EEB401DD
:100F82000280030210A2900055E0D394C7400B9058
:100F92000055E0C394C8F551801A900055E0D394EF
:100FA20063400B900055E0C39464F55180069000B5
:100FB20055E0F551E55175F002A4FFAEF08F74EFE4
:100FC2009000781270EBEFFCE0FDEC90007B127069
:100FD200EBEDFCE0FDEC2DB5510280030210930F06
:100FE200EF9000781270EBE574FFE0FCEF90007C6C
:100FF2001270EBECFFE0FCEFC39CB55102800302E0
:101002001093E57490007A1270EBE574FFE0FCEF48
:1010120090007D1270EBECFFE0FCEF2CB55172E515
:101022007490007E1270EBE0C395519008D4F0E505
:101032007490007F1270EBE0C395519008D5F0E5F3
:10104200749000821270EBE0C395519008D6F0E5DF
:10105200749000831270EBE0C395519008D7F0E5CD
:10106200749000841270EBE0C395519008D8F0E5BB
:10107200749000851270EBE0C395519008D9F0127C
:1010820006107599F97464F5097508001205E48073
:10109200FE7599FF7464F5097508001205E480FE77
:0F3C2A00020C5E020D41020E9E020F11020F5C92
:1010A20022E54E903C39F828287302118790088671
:1010B200E0FEA3E0FF900045120048E0F599900899
:1010C200861270C8900886E0FEA3E0FF741C6F4E83
:1010D2007003754E00021187856F9902118790087F
:1010E20086E0FEA3E0FF900078120048E0F599EF59
:1010F200B40107EEB40703754E009008861270C85B
:07110200021187900887E04D
:0F3C39000210AC0210AF0210DA0210E002110507
:10110900903CABF82828738553998067856099804E
:1011190062856299805D8566998058856899805352
:10112900856999804E856A998049856B9980449033
:101139000017E0F599803CA22DB340077599FAC2D2
:101149002D8017A222B3400575990F800B9000439B
:10115900E0F599900043E4F0C2228017856C9980EC
:1011690012856799800D856D9980087599FC8003B2
:03117900754E00B0
:103CAB0002111002111502111A02111F0211240226
:103CBB00112902112E021133021138021140021187
:0D3CCB006502116A02116F02117402117975
:0B117C009008861270C88003123F121A
:033C4800021184E2
:1011870022E538255BFFAE5A50010E900078120019
:1011970048E0F539E538255BFFAE5A50010E0FBF21
:1011A70000010E900078120048E0F53A85403CE5D2
:1011B70039B53A058539388041E53AD39539401D27
:1011C700E53AC39539853BF0A4FFAEF0E53C8E04C4
:1011D7008F05FF1270AAED2539F538801DE539C353
:1011E700953A853BF0A4FFAEF0E53C8E048F05FFF2
:1011F7001270AAEDF4042539F53822E53AD395396A
:10120700401DE53AC39539853BF0A4FFAEF0E53CB8
:101217008E048F05FF1270AAED2539F538801DE57C
:1012270039C3953A853BF0A4FFAEF0E53C8E048FB9
:1012370005FF1270AAEDF4042539F5382290007ED7
:10124700E0B4017FE56875F00A84FF7E008F38E51A
:101257006875F00A84ADF07C008D3B75400A755ABD
:1012670005755B24E538C394115005121188800673
:101277009005ADE0F538E538C394F05008E53890AF
:101287000067F0800674EF900067F0E56875F00A74
:1012970084FF7E008F38E56875F00A84ADF07C0026
:1012A7008D3B75400A755A05755B5AE538C394112D
:1012B700500512118880069005E3E0F538E538906F
:1012C700003EF02290007EE0B40102800302135931
:1012D700E56875F00A84FF7E008F38E56875F00AC7
:1012E70084ADF07C008D3B75400A755A05755B36F9
:1012F700E538C39411500512118880069005BFE0A8
:10130700F538E538C394F0500585384C8003754CA3
:10131700EFE56875F00A84FF7E008F38E56875F0A1
:101327000A84ADF07C008D3B75400A755A05755BE4
:1013370048E538C39411500512118880069005D1ED
:10134700E0F538E538C394F0500585384D800375CE
:101357004DEF22E56075F00484FF7E008F38E5606D
:1013670075F00484ADF07C008D3B754004755A011F
:10137700755B00E538C3943F5005121188800690CD
:1013870001B7E0F538E538900880F8E4F0E8A3F015
:10139700900042E075F020A4FFAEF09000C9E08E07
:1013A700048F05FF1270AA8D389000B1E0D39560C5
:1013B70050030214659000D5E0D395604010ED907E
:1013C70001B81270EBE0F52C752B00021462900047
:1013D700A0E0D395604043E5389001B81270EBE088
:1013E700F539E5389001D81270EBE0F53A9000D561
:1013F700E0F4042560F53B9000A0E0FE9000D5E006
:10140700F4042EF53CE539B53A05853938800312E1
:10141700120285382C752B008041E5389001D812CF
:1014270070EBE0F539E5389001F81270EBE0F53A2A
:101437009000A0E0F4042560F53B9000B1E0FE9039
:1014470000A0E0F4042EF53CE539B53A05853938B6
:10145700800312120285382C752B0002150C9000A0
:10146700D8E0D395605011E5389002381270EBE060
:10147700F52C752B0002150C9000A1E0D395605058
:1014870043E5389002181270EBE0F539E538900221
:10149700381270EBE0F53A9000A1E0F4042560F50E
:1014A7003B9000D8E0FE9000A1E0F4042EF53CE567
:1014B70039B53A05853938800312120285382C75FB
:1014C7002B008041E5389001F81270EBE0F539E523
:1014D700389002181270EBE0F53A9000B1E0F4048E
:1014E7002560F53B9000A1E0FE9000B1E0F4042EEA
:1014F700F53CE539B53A058539388003121202857E
:10150700382C752B00229000E9E0F53D75401175E8
:101517005A02755B00AE52AF53E53D75F00FA4FD5F
:10152700ACF0EDD39FEC9E4021E53D8E048F05FF87
:101537001270AAED75F010A4FFAEF0E56075F0111A
:1015470084FD7C00ED2FF53E800EE56075F011847B
:10155700FF7E00EF24F0F53E853E38E56075F0111B
:1015670084AFF07E008F3B12118885383FAE52AFB3
:10157700539000E9E075F00FA4FDACF0EDD39FECBC
:101587009E4028755A02755B10853E381211888572
:101597003F3985383AAE52AF53E53D8E048F05FF8C
:1015A7001270D58D3B853D3C121202E538900880BC
:1015B700F8E4F0E8A3F0752C64752B00229000E99D
:1015C700E0F53D754011755A02755B00AE52AF5399
:1015D700E53D75F00FA4FDACF0EDD39FEC9E4021E7
:1015E700E53D8E048F05FF1270AAED75F010A4FF7C
:1015F700AEF0E56275F01184FD7C00ED2FF53E80BD
:101607000EE56275F01184FF7E00EF24F0F53E854C
:101617003E38E56275F01184AFF07E008F3B121102
:101627008885383FAE52AF539000E9E075F00FA4BC
:10163700FDACF0EDD39FEC9E4028755A02755B1008
:10164700853E38121188853F3985383AAE52AF53F7
:10165700E53D8E048F05FF1270D58D3B853D3C120D
:101667001202E538900880F8E4F0E8A3F0E56C6032
:1016770017E56CC394FE50109000DDE0B4020990AA
:1016870000CBE0D3940B5002801F900880E0FEA3AC
:10169700E0FFE56C1270BA74E78E048F05FF1270D5
:1016A700AA900880ECF0A3EDF09000B3E0B4045FDB
:1016B700E56075F00484FF7E008F38E56075F004FF
:1016C70084ADF07C008D3B754004755A01755B0055
:1016D700E538C3943F500512118880069001B7E0A2
:1016E700F538900880E0FEA3E0FFE5381270BA7481
:1016F700328E048F05FF1270AA900880E0FEA3E0E7
:10170700FFEF2DFDEE3CFC900880ECF0A3EDF075AB
:101717002C64752B002290007EE0B40146E56875C5
:10172700F00A84FF7E008F38E56875F00A84ADF013
:101737007C008D3B75400A755A05755B00E538C31B
:10174700941150051211888006900589E0F538AE8E
:101757002BAF2CE5382FFF50010E74641270FD8EED
:101767002B8F2C90007FE0B40146E56975F00A8461
:10177700FF7E008F38E56975F00A84ADF07C008D37
:101787003B75400A755A05755B6CE538C394115073
:101797000512118880069005F5E0F538AE2BAF2CC1
:1017A700E5382FFF50010E74641270FD8E2B8F2CBD
:1017B70090008EE0B40249E56BC3944175F005844F
:1017C700FF7E008F38E56B75F00584ADF07C008DEA
:1017D7003B754005755A06755B00E538C394135091
:1017E70005121188800690068BE0F538AE2BAF2CDA
:1017F700E5382FFF50010E74641270FD8E2B8F2C6D
:101807009000D0E0B4020280030218BCE56075F0D6
:101817001584FF7E008F38E56075F01584ADF07C88
:10182700008D3B754015755A03755BF4E538C39415
:101837000B50051211888006900477E0F538E538DB
:1018470075F0FFA4FFAEF09000D1E08E048F05FF86
:101857001270AAED900063F0E56775F078A4FFAE0B
:10186700F074FF8E048F05FF1270AA8C5A8D5B747B
:10187700028C068D071200398F38AC5AAD5B7404A1
:10188700FF1270D58D3B754004755A06755B28E5C8
:1018970038C3941D500512118880069006BDE0F5E7
:1018A70038AE2BAF2CE5382FFF50010E7464127041
:1018B700FD8E2B8F2C90007DE0B4025DE56275F004
:1018C70064A4FFAEF074081200398E5C8F5D740556
:1018D7008E048F05FF1270AA8D38AE5CAF5D74055C
:1018E7008E048F05FF1270D58D3B754005755A051F
:1018F700755BDEE538C39413500512118880069096
:101907000669E0F538AE2BAF2CE5382FFF50010EF6
:1019170074641270FD8E2B8F2C9000BFE0707F9047
:101927000042E075F00A84FF7E008F38900042E0A5
:1019370075F00A84ADF07C008D3B75400A755A0539
:10194700755BC0E538C3940E500512118880069068
:101957000646E0F538E538900068F09000DEE0B420
:10196700023C900042E075F00A84FF7E008F3890B9
:101977000042E075F00A84ADF07C008D3B75400AAB
:10198700755A05755BCFE538C3940E50051211885B
:101997008006900655E0F538E538900069F022900A
:1019A7000086E0B401179008DBE0252CFFAE2B5032
:1019B700010E9000DAE01270FD8E2B8F2C9000FE46
:1019C700E0B401149000FFE0A852B800049553500A
:1019D70007E560C39561400280139000A8E0252CBD
:1019E700FFAE2B50010E8E2B8F2C021E0D90008602
:1019F700E0B40306A22AB3B3400280509008E5E0A2
:101A070070109008DEE0C39405A852B800069553FD
:101A1700400280109000A8E0252CFFAE2B50010E4D
:101A27008E2B8F2C9008E5E0600D9008DEE0A85221
:101A3700B800069553400280109000A8E0252CFFBF
:101A4700AE2B50010E8E2B8F2C021E0D900080E0C6
:101A5700B402028003021E0D900083E0602FE56848
:101A6700D39446402890000EE0FEA3E0FF9000BE0E
:101A7700E075F003A4FDACF0EFD39DEE9C400E9013
:101A870000E2E0A852B80005D395535003021E0D9B
:101A97009000B3E0B403028003021C5585625B75B6
:101AA7005A0090008AE0A852B800049553500E904F
:101AB700008BE0A85AB80005D3955B5003021C526F
:101AC700E56275F002A4FFAEF074158E048F05FF72
:101AD7001270AA8C068D07900608120048FEE0FFD8
:101AE700EE900082E0FEEF8E0088F0A4FFAEF07467
:101AF700648E048F05FF1270AA8C5A8D5B9000428A
:101B0700E075F018A4FFAEF09000C9E08E048F05D1
:101B1700FF1270AA8C068D07900620120048AE5A55
:101B2700AF5BE01270BA74648E048F05FF1270AA5F
:101B37008C5A8D5BE566A85AB80005D3955B5003B0
:101B4700021BC9E566C3955BFFE4955AFE8E5A8F63
:101B57005B7428BE00039F500C755B28755A007490
:101B67000D900043F0AE5AAF5B900083E01270BA5D
:101B770074288E048F05FF1270AA8C5A8D5B90080B
:101B870080E0FEA3E0FF740A8E048F05FF1270AA9F
:101B97008D068C07AC5AAD5BCFCECF120003740A0B
:101BA7008E048F05FF1270AA8C5A8D5B900880E017
:101BB700FEA3E0FF127105900880EEF0A3EFF0029C
:101BC7001C52E566A85AB80004955B507EAE5AAF22
:101BD7005BE5661270FD8E5A8F5B7428BE00039F0B
:101BE700500C755B28755A00740D900043F0AE5A7F
:101BF700AF5B900083E01270BA74288E048F05FFE4
:101C07001270AA8C5A8D5B900880E0FEA3E0FF74E7
:101C17000A8E048F05FF1270AA8D068C07AC5AAD89
:101C27005BCFCECF120003740A8E048F05FF1270AC
:101C3700AA8C5A8D5B900880E0FEA3E0FFEF2DFD94
:101C4700EE3CFC900880ECF0A3EDF0021E0D900036
:101C5700CBE08560F0A4FFAEF074051270BA74078C
:101C67001200398E5A8F5B90008AE0A852B80004A0
:101C77009553501290008BE075F002A4FDACF0EF85
:101C8700C39DEE9C4003021E0DE56075F00B84FFBB
:101C97007E00900608120048FEE0FFEE900082E00A
:101CA700FEEF8E0088F0A4FFAEF074648E048F05FB
:101CB700FF1270AA8C5A8D5B900042E075F018A451
:101CC700FFAEF09000C9E08E048F05FF1270AA8C5A
:101CD700068D07900620120048AE5AAF5BE01270DF
:101CE700BA74648E048F05FF1270AA8C5A8D5BE557
:101CF70066A85AB80005D3955B5003021D84E566B4
:101D0700C3955BFFE4955AFE8E5A8F5B7428BE001D
:101D1700039F500C755B28755A00740D900043F0B3
:101D2700AE5AAF5B900083E01270BA74288E048FAE
:101D370005FF1270AA8C5A8D5B900880E0FEA3E025
:101D4700FF740A8E048F05FF1270AA8D068C07ACEC
:101D57005AAD5BCFCECF120003740A8E048F05FFF6
:101D67001270AA8C5A8D5B900880E0FEA3E0FF12E8
:101D77007105900880EEF0A3EFF0021E0DE566A84E
:101D87005AB80004955B507EAE5AAF5BE566127099
:101D9700FD8E5A8F5B7428BE00039F500C755B281D
:101DA700755A00740D900043F0AE5AAF5B900083F4
:101DB700E01270BA74288E048F05FF1270AA8C5A2D
:101DC7008D5B900880E0FEA3E0FF740A8E048F0508
:101DD700FF1270AA8D068C07AC5AAD5BCFCECF121F
:101DE7000003740A8E048F05FF1270AA8C5A8D5B4C
:101DF700900880E0FEA3E0FFEF2DFDEE3CFC90088D
:101E070080ECF0A3EDF0229000DEE0B4027BE56009
:101E170075F00884FF7E008F38E56075F00884ADA3
:101E2700F07C008D3B754008755A01755BE0E5381D
:101E3700C3943F50051211888006900277E0F53869
:101E4700E538900882F8E4F0E8A3F0900882E0FE15
:101E5700A3E0FFAC2BAD2C12000374648E048F0536
:101E6700FF1270AA900882ECF0A3EDF090007BE0DF
:101E77008C068D071270BA74648E048F05FF12707A
:101E8700AA900882ECF0A3EDF0900880E0FEA3E0B2
:101E9700FFAC2BAD2C12000374648E048F05FF1268
:101EA70070AA900880ECF0A3EDF090007BE08C0620
:101EB7008D071270BA74648E048F05FF1270AA9092
:101EC7000880ECF0A3EDF0A204401DAE52AF5374AE
:101ED70005BE00039F5002D204E562D394CC4008AC
:101EE700D2027411900043F0229000DDE0B40208A2
:101EF7009000CBE0640B60028045900880E0FEA371
:101F0700E0FFE56C1270BA74E78E048F05FF12705C
:101F1700AA900880ECF0A3EDF09000DEE0B4021F79
:101F2700900882E0FEA3E0FFE56C1270BA74E78EBA
:101F3700048F05FF1270AA900882ECF0A3EDF090D1
:101F4700009DE05402601B900094E0A852B8001274
:101F5700D39553400DA204B3B35007E562C3949AD7
:101F67004002805FAE35AF36900092E075F002A474
:101F7700FDACF0EF2DFDEE3CFC74022DFD50010C85
:101F8700E562BC003ED39D403A754401A23140331F
:101F9700900093E075F05EA4FDACF07405FF12703D
:101FA700AA8C5C8D5D124A8E900880E0FEA3E0FF4C
:101FB700900093E02FFF50010E900880EEF0A3EF02
:101FC700F0D231E562A835B8000495365002C23127
:101FD700856236753500E54470030220E69000F00F
:101FE700E0C3954450030220D8900100E0C3940257
:101FF7004003022082E56875F00A84FF7E009005A1
:1020070078120048E0F55B755A00AE5AAF5B900056
:1020170093E01270BA74648E048F05FF1270AA8C55
:102027005C8D5D9000F0E004C395448C068D07122B
:1020370070BA9000F0E08E048F05FF1270AA8C5CD6
:102047008D5D900880E0FEA3E0FFEF2DFDEE3CFCE8
:10205700900880ECF0A3EDF09000DEE0B4021A9057
:102067000882E0FEA3E0FFAA5CAB5DEF2BFBEE3A34
:10207700FA900882EAF0A3EBF080569000F0E004B3
:10208700C39544854CF0A4FFAEF09000F0E08E04B9
:102097008F05FF1270AA8C5C8D5D900880E0FEA30F
:1020A700E0FFEF2DFDEE3CFC900880ECF0A3EDF097
:1020B7009000DEE0B4021A900882E0FEA3E0FFAAD7
:1020C7005CAB5DEF2BFBEE3AFA900882EAF0A3EBEC
:1020D700F005449000F0E0C3954450037544009028
:1020E700009DE05401601B900091E0A852B80012D7
:1020F700D39553400DA204B3B35007E560C394CC06
:102107004002806090008FE075F003A4FFAEF0E519
:10211700412FFF50010E74032FFF50010EE560BEE3
:102127000042D39F403E754501A231403790009051
:10213700E075F05EA4FFAEF074058E048F05FF1204
:1021470070AA8C5C8D5D124A8E900880E0FEA3E039
:10215700FF900090E02FFF50010E900880EEF0A353
:10216700EFF0D231E560C395415002C2318560413D
:10217700E54570030222809000F1E0C395455003C6
:10218700022272900100E0C39402400302221CE580
:102197006875F00A84FF7E00900578120048E0F524
:1021A7005B755A00AE5AAF5B900090E01270BA743C
:1021B700648E048F05FF1270AA8C5C8D5D9000F110
:1021C700E004C395458C068D071270BA9000F1E0C4
:1021D7008E048F05FF1270AA8C5C8D5D900880E0DD
:1021E700FEA3E0FFEF2DFDEE3CFC900880ECF0A392
:1021F700EDF09000DEE0B4021A900882E0FEA3E062
:10220700FFAA5CAB5DEF2BFBEE3AFA900882EAF08F
:10221700A3EBF080569000F1E004C39545854DF09F
:10222700A4FFAEF09000F1E08E048F05FF1270AAB4
:102237008C5C8D5D900880E0FEA3E0FFEF2DFDEE46
:102247003CFC900880ECF0A3EDF09000DEE0B402D7
:102257001A900882E0FEA3E0FFAA5CAB5DEF2BFBC0
:10226700EE3AFA900882EAF0A3EBF005459000F108
:10227700E0C395455003754500900880E0FEA3E054
:10228700FF9000A2E0BE00039F500D9000A2E090D7
:102297000880F8E4F0E8A3F09000DEE0B4021290C2
:1022A7000882E0FEA3E0FF9000A2E0BE00059F4089
:1022B70002800D9000A2E0900882F8E4F0E8A3F015
:1022C700229000DEE0B401028003022416A204B3C8
:1022D70050030223FD9000A9E0B4017A900880E042
:1022E700FEA3E0FFAC52AD53120003743C8E048F83
:1022F70005FF1270AA9000B9E0BC00159D4012902E
:102307000880E0FEA3E0FF9000BBE0BE00039F5003
:1023170002D203900880E0FEA3E0FFAC52AD531257
:102327000003743C8E048F05FF1270AA9000B9E079
:10233700C3940ABC001AD39D4016900880E0FEA300
:10234700E0FF9000BBE0C39405BE0004D39F50029A
:102357008002C203807A900880E0FEA3E0FFAC52BF
:10236700AD5312000374788E048F05FF1270AA9084
:1023770000B9E0BC00159D4012900880E0FEA3E084
:10238700FF9000BBE0BE00039F5004D20380419042
:102397000880E0FEA3E0FFAC52AD5312000374784F
:1023A7008E048F05FF1270AA9000B9E0C3940ABC8F
:1023B700001AD39D4016900880E0FEA3E0FF90002E
:1023C700BBE0C39405BE0004D39F50028002C20342
:1023D700A203B34021900880E0FEA3E0FF9000BA7B
:1023E700E01270BA74648E048F05FF1270AA900809
:1023F70080ECF0A3EDF0A203B3400CA235400674C5
:1024070024900043F0D235A2034002C2358002C2B5
:102417000390003EE06006A204B3B3400280199027
:102427000880E0FEA3E0FF90003EE02FFF50010E82
:10243700900880EEF0A3EFF0A201B34006A202B32A
:10244700B35009900016E4F0A3F0802D900880E0C7
:10245700FEA3E0FF7400D39F74019E401190088093
:10246700E0F8A3E0900016C8F0A3C8F0800B74FF53
:10247700900016F8E4F0E8A3F09000C0E0C39404DD
:10248700400C9008E2E0C3940240030225709000DC
:10249700A9E0B40147900880E0FEA3E0FF745E1254
:1024A70070BA74058E048F05FF1270AA900880EC2D
:1024B700F0A3EDF09000DEE0B4021F900882E0FE8A
:1024C700A3E0FF745E1270BA74058E048F05FF12C5
:1024D70070AA900882ECF0A3EDF08045900880E0A8
:1024E700FEA3E0FF745E1270BA740A8E048F05FFB4
:1024F7001270AA900880ECF0A3EDF09000DEE0B433
:10250700021F900882E0FEA3E0FF745E1270BA74A7
:102517000A8E048F05FF1270AA900882ECF0A3EDD3
:10252700F0900880E0FEA3E0FF7402BE000CD39F8A
:102537004008752A02752900800A900880E0F5296D
:10254700A3E0F52A900882E0FEA3E0FF7402BE0034
:102557000CD39F4008752E02752D00800A900882C3
:10256700E0F52DA3E0F52E8046900880E0FEA3E07D
:10257700FF7401BE000CD39F4008752A017529001E
:10258700800A900880E0F529A3E0F52A900882E008
:10259700FEA3E0FF7401BE000CD39F4008752E0117
:1025A700752D00800A900882E0F52DA3E0F52E90A6
:1025B7000014E529F0A3E52AF0A238B34009C201C7
:1025C700900016E4F0A3F022900042E09003781206
:1025D70070EBE0F542754364900042E0FE9000B472
:1025E700E0D39E4037E56075F00884FF7E008F38A2
:1025F700E56075F00884ADF07C008D3B754008758B
:102607005A03755B96E538C3941F500512118880ED
:102617000690042DE0F5388538438035E56075F080
:102627000884FF7E008F38E56075F00884ADF07C84
:10263700008D3B754008755A03755BB6E538C39442
:102647001F5005121188800690044DE0F538853833
:1026570043229000EAE0F53D754011755A04755B19
:1026670000AE52AF53E53D75F00FA4FDACF0EDD3CE
:102677009FEC9E4021E53D8E048F05FF1270AAED69
:1026870075F010A4FFAEF0E56075F01184FD7C00D5
:10269700ED2FF53E800EE56075F01184FF7E00EFAB
:1026A70024F0F53E853E38E56075F01184AFF07E85
:1026B700008F3B12118885383FAE52AF539000EA26
:1026C700E075F00FA4FDACF0EDD39FEC9E402875AC
:1026D7005A04755B10853E38121188853F39853855
:1026E7003AAE52AF53E53D8E048F05FF1270D58D7C
:1026F7003B853D3C121202853842754364229000A7
:10270700EAE0F53D754011755A04755B00AE52AFAE
:1027170053E53D75F00FA4FDACF0EDD39FEC9E4063
:1027270021E53D8E048F05FF1270AAED75F010A408
:10273700FFAEF0E56275F01184FD7C00ED2FF53EEC
:10274700800EE56275F01184FF7E00EF24F0F53E00
:10275700853E38E56275F01184AFF07E008F3B123D
:10276700118885383FAE52AF539000EAE075F00FFD
:10277700A4FDACF0EDD39FEC9E4028755A04755B21
:1027870010853E38121188853F3985383AAE52AFE9
:1027970053E53D8E048F05FF1270D58D3B853D3C7B
:1027A7001212028538427543649000E5E0B404795B
:1027B700900042E0FE9000B4E0D39E4037E560759C
:1027C700F00884FF7E008F38E56075F00884ADF06F
:1027D7007C008D3B754008755A03755B96E538C3D9
:1027E700941F5005121188800690042DE0F5388556
:1027F70038438035E56075F00884FF7E008F38E543
:102807006075F00884ADF07C008D3B754008755A03
:1028170003755BB6E538C3941F500512118880060F
:1028270090044DE0F5388538432290007EE0B401EE
:102837003BE56875F00A84FF7E008F38E56875F020
:102847000A84ADF07C008D3B75400A755A05755BAF
:1028570012E538C394115005121188800690059B24
:10286700E0F538E5432538C39464F54390007FE0ED
:10287700B4013BE56975F00A84FF7E008F38E5698E
:1028870075F00A84ADF07C008D3B75400A755A05DA
:10289700755B7EE538C39411500512118880069048
:1028A7000607E0F538E5432538C39464F543E54268
:1028B7002543F537900086E0B402109008DAE0254A
:1028C70037FE9000DAE0F4042EF5379000DDE0D310
:1028D70094014040E56CC394E7501D74E7C3956CC1
:1028E700FE9008DCE08E00F5F0E884FF7E008F386C
:1028F700E5372538F537801CE56CC394E7FE90086B
:10290700DCE08E00F5F0E884FF7E008F38E537C302
:102917009538F537A2044006E5422464F537E537D4
:10292700D394644009E537C39464F537800375375A
:10293700009000B6E0C3953750069000B6E0F53733
:1029470022D201900066E0A852B800049553503E89
:10295700900066E0A852B800049553500375370FEE
:10296700900066E004A852B80004955350037537E9
:1029770007900066E02402A852B80004955350025D
:10298700C201900066E060067409900043F0C2300F
:102997007E017F009000BCE01270BA9000CBE08E01
:1029A700048F05FF1270AAE560BC000CD39D400898
:1029B700D238740A900043F090007EE0B401099089
:1029C70000BDE0C39568400280159000CFE0A85293
:1029D700B8000495535002C201740B900043F09065
:1029E700007EE0B40107E568C394644002801D904F
:1029F7000115E0600D900115E0A852B80006955347
:102A070040028008C201740B900043F0A20140030A
:102A1700753700C2379000FEE0B401149000FFE064
:102A2700A852B8000495535007E560C3956140026A
:102A3700802A9000A7E0D3941D400B9000A7E0C325
:102A4700941EF5378003753700A23440087415903B
:102A57000043F0D237D234D232022B42C232C234D0
:102A6700900086E0B40306A22AB3B34003022B42C8
:102A77009008DEE0C39405A852B8000495535006A9
:102A87009008E5E06002801F9000A7E0D3941D4006
:102A97000B9000A7E0C3941EF537800375370074C9
:102AA7000C900043F0D2379008DEE0A852B800043B
:102AB700955350069008E5E07002801F9000A7E04C
:102AC700D3941D400B9000A7E0C3941EF5378003F5
:102AD700753700740C900043F0D2379008DEE0A8F9
:102AE70052B80004955350319000C5E0B40228D283
:102AF700309008E4E0FE9008E5E0D39E5006900889
:102B0700E5E0700280099008E4E4F0C230800690A6
:102B170008E4E004F08002C2019008DEE02405A882
:102B270052B80004955350139000C5E0B4020A90C0
:102B370008E5E07002D2308002C201A22FB340271D
:102B47009000A7E0D3941D400B9000A7E0C3941E0C
:102B5700F5378003753700A23340067410900043A1
:102B6700F0D233D2378002C23385376D9000A7E0A9
:102B7700D3941D4018900075E02537FE900042E081
:102B870075F01E84FC7F00EE2CF5378029A237B341
:102B97004008900075E0F537801C900077E02537F6
:102BA700FE900075E02EFE900042E075F01E84FC5A
:102BB7007F00EE2CF537A238B34005D230756D0093
:102BC70022900042E075F00584FF7E008F38900068
:102BD70042E075F00584ADF07C008D3B75400575CE
:102BE7005A03755BD69000C9E01475F00584FF7E23
:102BF70000E538BE00039F5005121188800BE538A9
:102C070090044E1270EBE0F538E5389008DDF0904F
:102C170008DDE0FE9000B8E0C39E50089000B8E0E1
:102C27009008DDF09000A7E0D3941D401E9008DDCA
:102C3700E0FE900075E02EFE900042E075F01E84E5
:102C4700FC7F00EE2C9008DDF08031A237B3400AFC
:102C5700900075E09008DDF080229008DDE0FE909E
:102C67000077E02EFE900075E02EFE900042E075A2
:102C7700F01E84FC7F00EE2C9008DDF02290007E91
:102C8700E0B40136E56875F00A84FF7E00900578A8
:102C9700120048E0F547E547D394644010E547C381
:102CA700946475F00F84FF7E008F4780037547009B
:102CB70090009BE02547F547800690009BE0F5478D
:102CC70022E56875F00A84FF7E00900578120048B7
:102CD700E0C394694007E568D3946440559000E5E4
:102CE700E0C39403502690087AE0FEA3E0FF740443
:102CF700120039E5601270BA740F8E048F05FF1247
:102D070070AA900878ECF0A3EDF0802490087AE0A0
:102D1700FEA3E0FF7404120039E5621270BA740F63
:102D27008E048F05FF1270AA900878ECF0A3EDF0DF
:102D3700800F90087AE0F8A3E0900878C8F0A3C85D
:102D4700F0A204401A90087AE0FEA3E0FF74031291
:102D570070BA7401120039900878EEF0A3EFF09082
:102D6700008EE0B40262E56BC3944175F00584FF01
:102D77007E008F38E56B75F00584ADF07C008D3BE8
:102D8700754005755A06755B14E538C394175005E9
:102D9700121188800690069FE0F538900878E0FECB
:102DA700A3E0FF740A8E048F05FF1270AAE5388C22
:102DB700068D071270BA740A8E048F05FF1270AA67
:102DC700900878ECF0A3EDF0900878E0FEA3E0FF20
:102DD70090087EE0FCA3E0FDEDD39FEC9E400F90B2
:102DE700087EE0F8A3E0900878C8F0A3C8F022E5D1
:102DF7000875F004A4FFAEF09006BB120048E090FF
:102E07003C4BF8282873804C85537480479000CB3F
:102E1700E08560F0A4FFAEF074081200398F74806B
:102E270033856274802E856874802985697480244F
:102E3700856A74801F856B74801A856C748015850C
:102E470067748010856674800B856D7480069000AA
:042E570017E0F57417
:103C4B00022E0D022E0F022E14022E28022E2D02F2
:103C5B002E32022E37022E3C022E41022E46022E0F
:073C6B004B022E50022E5502
:102E5B00E50875F004A4FFAEF09006BC120048E53F
:102E6B000875F004A4FFAEF0E0FC9006BD1200481C
:102E7B00ECFEE0FFEEC39F4003022F63E50875F005
:102E8B0004A4FFAEF09006BB120048E0B40441E589
:102E9B000875F004A4FFAEF09006BD120048E0C325
:102EAB009574500AE508F50CD39239123DF0E508FC
:102EBB0075F004A4FFAEF09006BC120048E0D39569
:102ECB0074400AE508F50CC39239123DF0022F61EC
:102EDB00E50875F004A4FFAEF09006BC120048E0C4
:102EEB00C395745015E50875F004A4FFAEF0900679
:102EFB00BD120048E0D395745002800AE508F50C2A
:102F0B00D39239123DF0E50875F004A4FFAEF090B2
:102F1B0006BC120048E0D395745015E50875F00413
:102F2B00A4FFAEF09006BD120048E0C39574500AA2
:102F3B00E508F50CC39239123DF09006C3E0B401DD
:102F4B00099000D7E0D395625002800A7402F50C09
:102F5B00C39239123DF0806AE50875F004A4FFAE08
:102F6B00F09006BC120048E0D395744015E5087547
:102F7B00F004A4FFAEF09006BD120048E0C39574B8
:102F8B004002800AE508F50CC39239123DF0E508C2
:102F9B0075F004A4FFAEF09006BC120048E0C39598
:102FAB00744015E50875F004A4FFAEF09006BD1251
:102FBB000048E0D39574400AE508F50CD39239121A
:102FCB003DF022AE2FAF3074C9BE000CD39F40082A
:102FDB00782F12710D0230E8753001752F00AE524B
:102FEB00AF53E547BE000DD39F40099000ADE0D332
:102FFB00954840028023754800E547C39553F57407
:10300B009000B0E0D395464008E5462574F5468020
:10301B00069000B0E0F54680020548900089E0D3A9
:10302B009562401CE560C395614015AE52AF53E508
:10303B0047BE00039F50099000AEE0D39549400274
:10304B00806E9008DFE0A852B800049553500375CA
:10305B004B009008DFE0A852B8000BD39553400605
:10306B00E5539008DFF0E54B7041E553C39547F509
:10307B0074E574D3940540037574059000AFE0C3F9
:10308B0095465007E574C3954640028009E546C353
:10309B009574F54680069000AFE0F5469000AFE0E2
:1030AB00D3954640069000AFE0F546754900800287
:1030BB000549E54B7016900089E0C39562500DE50C
:1030CB00472405A852B8000695534002800F900084
:1030DB009CE0F546754B0174789008DFF022AE2F1B
:1030EB00AF3074E9D39F74039E4008782F12710D93
:1030FB0002328F753001752F00754632A22B402A94
:10310B0075461990009CE075F002A4FFAEF0E548FF
:10311B00BE0006D39F4002D22B0548754B03747833
:10312B009008DFF0754A00023276AE52AF53E54796
:10313B006F4E7003023276E547BE000DD39F4009F8
:10314B009000ADE0D395484002800F754800E54BE9
:10315B00C394035003754619800DE547C39553F58A
:10316B0074E5482574F548900089E0D39562400ECC
:10317B009008DFE0A852B80007D395534002800CAB
:10318B00054A90009CE0B54A03754B00E54BB40330
:10319B0006A204B3B34002800A054AE54AB43C03D5
:1031AB00754B02E54BB402299008DFE0A852B8003A
:1031BB000ED395534009E5539008DFF0754A009004
:1031CB000089E0C395625009754A0074789008DF56
:1031DB00F0E54B705A900089E0D39562401CE56096
:1031EB00C395614015AE52AF53E547BE00039F50E8
:1031FB00099000AEE0D395494002800875490075EF
:10320B00464B8028E553C39547F574E574D3940575
:10321B004003757405900089E0D395624008E54939
:10322B002574F5498006E5492406F549754A00E5FC
:10323B004B7016900089E0C39562500DE54724054D
:10324B00A852B80006955340028003754B01E54B1D
:10325B00B40118754619054A90009CE0B54A0675ED
:10326B004B02754A0074789008DFF0A202B340035A
:10327B00754632E54675F00AA4FFAEF0900884EE71
:10328B00F0A3EFF022E570903C72F8282873023C13
:10329B000B900081E070030235BA9000B7E0B401E7
:1032AB00028003023450900040E0655F6009E553F3
:1032BB004552600302344D7E017F00E5BE1270BAA9
:1032CB00E5BD2FFF50010E8E5A8F5B9000B5E0B419
:1032DB00461B740E1270BA900065E08E048F05FFCA
:1032EB001270AA900888ECF0A3EDF0801DAE5AAFD7
:1032FB005B74101270BA900065E08E048F05FF129C
:10330B0070AA900888ECF0A3EDF0E56C600FE56C0B
:10331B00C394FE50089000DDE0640260028064906C
:10332B0000CBE0B40B1F900888E0FEA3E0FF74E72E
:10333B001270BAE56C8E048F05FF1270AA90088884
:10334B00ECF0A3EDF09000CBE0D3940B4008900091
:10335B00B3E064046002802B900888E0FEA3E0FFDA
:10336B0090088CE0FCA3E0FDEFD39DEE9C400D128A
:10337B007105900888EEF0A3EFF08007900888E4C1
:10338B00F0A3F0900888E0FEA3E0FFEFD39400EEEB
:10339B0094014008D2387426900043F0A238B3B39E
:1033AB00502C7E057F009000CBE08E048F05FF1222
:1033BB0070AA900888E0FEA3E0FFEFC39DEE9C404F
:1033CB000FAC52AD53740FBC0004D39D500280025E
:1033DB00C238900081E0B4022790088AE0FEA3E097
:1033EB00FF900888E0FCA3E0FDEF2DFDEE3CFC74A4
:1033FB00018C068D07120039900888EEF0A3EFF0D0
:10340B00900888E0FEA3E0FF90088AE0FCA3E0FDB3
:10341B00EDD39FEC9E4004D22E8002B22E900888F2
:10342B00E0F8A3E090088AC8F0A3C8F09000B3E0DE
:10343B0064016006A22EB3B340028006900889E0B7
:10344B00F5600235B8D22E7E017F00E5BE1270BA50
:10345B00E5BD2FFF50010E8E5A8F5B9000B5E0B487
:10346B00461B740E1270BA900065E08E048F05FF38
:10347B001270AA900888ECF0A3EDF0801DAE5AAF45
:10348B005B74101270BA900065E08E048F05FF120A
:10349B0070AA900888ECF0A3EDF0E56C600FE56C7A
:1034AB00C394FE50089000DDE064026002806490DB
:1034BB0000CBE0B40B1F900888E0FEA3E0FF74E79D
:1034CB001270BAE56C8E048F05FF1270AA900888F3
:1034DB00ECF0A3EDF09000CBE0D3940B4008900000
:1034EB00B3E064046002802B900888E0FEA3E0FF49
:1034FB0090088CE0FCA3E0FDEFD39DEE9C400D12F9
:10350B007105900888EEF0A3EFF08007900888E42F
:10351B00F0A3F0900888E0FEA3E0FFEFD39400EE59
:10352B0094014008D2387426900043F0A238B3B30C
:10353B00502C7E057F009000CBE08E048F05FF1290
:10354B0070AA900888E0FEA3E0FFEFC39DEE9C40BD
:10355B000FAC52AD53740FBC0004D39D50028002CC
:10356B00C238900081E0B4022790088AE0FEA3E005
:10357B00FF900888E0FCA3E0FDEF2DFDEE3CFC7412
:10358B00018C068D07120039900888EEF0A3EFF03E
:10359B00900888E0F8A3E090088AC8F0A3C8F090E0
:1035AB0000B3E064016006900889E0F56080037564
:1035BB00600090007DE0700675700302329075BB61
:1035CB0018023C0B023C0B90007DE070030237436A
:1035DB007E017F00E5BE1270BAE5BD2FFF50010ED4
:1035EB008E5A8F5B9000C3E0B4010F7E0F7FFFAC50
:1035FB005AAD5B1271058E5A8F5B9000E8E0B402F6
:10360B0045AE5AAF5B900020E0FCA3E0FDEDD39FED
:10361B00EC9E400A900020E55AF0A3E55BF0AE5A11
:10362B00AF5B900022E0FCA3E0FDEFD39DEE9C404E
:10363B000A900022E55AF0A3E55BF0AE5AAF5B743B
:10364B00041200398F629000E8E0704CAE5AAF5B09
:10365B00900020E0FCA3E0FDEFD39DEE9C4009120F
:10366B0071058E5A8F5B8006755B00755A00AE5ADA
:10367B00AF5B74101270BA9000E7E08E048F05FFF9
:10368B001270AA8C5A8D5B74FFBC0009D39D400548
:10369B00855B6280037562FE9000B3E0B40102802B
:1036AB0003023741A204B3B3500E900087E0A85237
:1036BB00B80005D39553500280719000C4E0856229
:1036CB00F0A4FFAEF074648E048F05FF1270AA8C09
:1036DB005A8D5BE56C6016E56CC394FE500F900041
:1036EB00DDE0B402089000CBE0640B60028017AE03
:1036FB005AAF5B74E71270BAE56C8E048F05FF123C
:10370B0070AA8C5A8D5BAE5AAF5B900888E0FCA315
:10371B00E0FDEDD39FEC9E4005855B60800BA22EF8
:10372B00B34006900889E0F560800BA22EB34006EB
:10373B00900889E0F5608003756200900080E0706E
:10374B000675700502329075BB19023C0B023C0BDF
:10375B00900080E070030237FBE55FD3955E40037A
:10376B000237F990001EE0FEA3E0FFE5661270FD44
:10377B0090001EEEF0A3EFF07E017F00E5BE12700D
:10378B00BAE5BD2FFF50010E8E5A8F5B9000EDE016
:10379B007013740A1270BA74518E048F05FF127075
:1037AB00AA8D668019AE5AAF5B740A1270BA8F0479
:1037BB008E057E017F95CDCCCD126FA88F66E56609
:1037CB00D39464400375666490001EE0FEA3E0FF93
:1037DB00E5662FFF50010E90001EEEF0A3EFF09068
:1037EB000084E0048E048F05FF1270AA8D6680039F
:1037FB007566329000D0E0700675700702329075D6
:10380B00BB13023C0B023C0B9000D0E0604A7E01E4
:10381B007F00E5BE1270BAE5BD2FFF50010E8E5A28
:10382B008F5B74041200398F679000D2E08567F0CC
:10383B00A4FDACF07464FF1270AA8D679000D1E008
:10384B008567F0A4FFAEF074FF8E048F05FF127036
:10385B00AAED900064F0800375670090007EE07025
:10386B000675700902329075BB17023C0B023C0BBC
:10387B0090007EE0B40102800302390F7E017F00CD
:10388B00E5BE1270BAE5BD2FFF50010E8E5A8F5B4D
:10389B009008E0E060199008E0E014906A9A12003A
:1038AB008CE493FC740193FDEDC39FEC9E4002806E
:1038BB00069008E0E014F09008E0E0C394B3501DCC
:1038CB00AE5AAF5B9008E0E004906A9A12008CE469
:1038DB0093FC740193FDEFC39DEE9C400280069018
:1038EB0008E0E004F09008E0E0FE9000A4E08E0019
:1038FB0088F0A4FFAEF074648E048F05FF1270AADB
:10390B008D68800375680090007FE0700675700B02
:10391B0002329075BB16023C0B023C0B90007FE011
:10392B00B4010280030239BB7E017F00E5BE127039
:10393B00BAE5BD2FFF50010E8E5A8F5B9008E1E068
:10394B0060199008E1E014906C0412008CE493FC75
:10395B00740193FDEDC39FEC9E400280069008E13D
:10396B00E014F09008E1E0C394B3501DAE5AAF5B86
:10397B009008E1E004906C0412008CE493FC740159
:10398B0093FDEFC39DEE9C400280069008E1E0049E
:10399B00F09008E1E0FE9000AAE08E0088F0A4FF12
:1039AB00AEF074648E048F05FF1270AA8D698003CC
:1039BB0075690075BB1F023C0B023C0B7E017F003F
:1039CB00E5BE1270BAE5BD2FFF50010E8E5A8F5B0C
:1039DB0074091270BA74E68E048F05FF1270AA8DEB
:1039EB006B900086E0700675700F02329075BB15F8
:1039FB00023C0B023C0B900086E07003023B527EB4
:103A0B00017F00E5BE1270BAE5BD2FFF50010E8E8F
:103A1B005A8F5B74041200398F6A900086E0B401F0
:103A2B00159000DAE0856AF0A4FFAEF0740712007F
:103A3B0039EF9008DBF0900086E0B402159000DAC5
:103A4B00E0856AF0A4FFAEF07407120039EF90081E
:103A5B00DAF0900086E0B403028003023B3590005D
:103A6B00C7E07052E56AC39419500FD22A9000A692
:103A7B00E09008DEF09008E3E4F0E56AD39464404C
:103A8B0004A22A4002802D9008E3E004F09008E3A2
:103A9B00E0FE900119E0B5060B9008DEE004F09013
:103AAB0008E3E4F09008DEE064966006900119E00C
:103ABB007002C22A80639000A6E070349000DAE0B6
:103ACB00856AF0A4FFAEF074FF8E048F05FF1270B1
:103ADB00AAED9008DEF0AE52AF53741EBE0006D3B3
:103AEB009F4002D22AE562D394E54002C22A802984
:103AFB00E56AC3940A500DAE52AF53741EBE000458
:103B0B00D39F50028002D22AE562D394E54002C2D1
:103B1B002A9000A6E09008DEF09008DEE0C3940542
:103B2B00500674059008DEF0C22F900086E0B404B6
:103B3B0014E56AC394195002D22FE56AD39432402C
:103B4B0002C22FC22A8003756A009000DDE0700666
:103B5B0075701102329075BB14023C0B023C0B903A
:103B6B0000DDE07003023BF87E017F00E5BE1270C2
:103B7B00BAE5BD2FFF50010E8E5A8F5B900102E00C
:103B8B007025EFD39421EE940E4005756CFF8015D4
:103B9B00AE5AAF5B74101270BA74E38E048F05FFCC
:103BAB001270AA8D6C8027AE5AAF5BEFD39449EE9F
:103BBB0094064005756CFF8015AE5AAF5B741012FE
:103BCB0070BA74638E048F05FF1270AA8D6CE56C4E
:103BDB0075F00BA4FFAEF09000CBE08E048F05FFC9
:103BEB001270AA90088CECF0A3EDF08003756C00BA
:103BFB00900081E0600575BB1A800375BB188000CF
:103C720002329902329C0235CF0235D20237580203
:103C8200375B02381002381302387802387B023967
:103C9200240239270239C40239C70239FE023A0125
:093CA200023B67023B6A023C0B85
:103C0B00E57075F00284AFF07E00EF4E7002D2ECDF
:033C1B000570220F
:0970EB002582F582500205832282
:0F008C0025E050020583258250020583F582226C
:10708900EF2F500205832582F582E5833E2EF58395
:0170990022D4
:1070FD00CFC39FFF50011E22C3EF9DFFEE9CFE22CA
:08710D000806B6000218062274
:0D70C800A3E004F070061270E1E004F02275
:0E003900048007C3CE13CECF13CFD5E0F6223E
:106FA800BC000FBE0008ED8FF084FFADF022E4FEB8
:106FB800FF22BE000DEF60FE54F0606F20E7030271
:106FC800705EEAC0E0EBC0E078017A0075F001EE8F
:106FD80020E710EF25E0FFEE33FE0AC5F023C5F0E9
:106FE80030E7F0EA5407F9096A7A007B0060010883
:106FF800C3EC9E40167004ED9F4010ED9FFDEC9E83
:10700800FCE5F0CA4ACA03F5F08005E5F003F5F09F
:10701800C3EE13FEEF13FFD9D77908CACBCAD8D06D
:10702800EAFEEBFFD0E0FBD0E0FA22EC8FF084FC24
:10703800ED54F045F0C48FF084FEEDC454F045F0F3
:10704800C48FF084FDEEC4FE54F02DFFEE540F3CC7
:10705800FEADF07C0022790078008FF0EC7E0820ED
:10706800E70DC3CD33CD33C933C9C833C8DEF08487
:1070780049F9E5F08FF0BE00E6FD7C00E9FFE8FE87
:0170880022E5
:0E70BA00F88FF0A4FFE5F0CE88F0A42EFE22A1
:10000300EF8DF0A4F9A8F0EF8CF0A428F8EE8DF0B2
:06001300A428FEE9FF2213
:10709A00600D782B0270A4007830D8FED5E0F82273
:1070AA00EEC0E07E00126FA8EFFDEEFCD0E0FE22FB
:0C70D500EEC0E07E00126FA8D0E0FE22AA
:03001B0002001EC2
:0300530002005652
:03009B00020071EF
:030000000270F497
:0970F40075817675D000024BF79E
:0B004800E5822FF582E5833EF5832260
:0A70E1000582D58202158315822274
:10001E00C0E0C0F0C083C082C0D075D000124B616A
:0B002E00D0D0D082D083D0F0D0E032E0
:10005600C0E0C0F0C083C082C0D075D000124B642F
:10006600D0D0D082D083D0F0D0E032C0E0C0F0C093
:1000760083C082C0D075D000124BB9D0D0D082D008
:0600860083D0F0D0E0324F
:00000001FF
